; Listing generated by Microsoft (R) Optimizing Compiler Version 15.00.21022.08 

	TITLE	c:\Develop\DScaler423a\DScaler\xml_prolog.tab.cpp
	.686P
	.XMM
	include listing.inc
	.model	flat

INCLUDELIB OLDNAMES

PUBLIC	?yynerrs@@3HA					; yynerrs
PUBLIC	?yychar@@3HA					; yychar
PUBLIC	?yylval@@3TYYSTYPE@@A				; yylval
PUBLIC	??_C@_1BK@ECDIFIKG@?$AAs?$AAy?$AAn?$AAt?$AAa?$AAx?$AA?5?$AAe?$AAr?$AAr?$AAo?$AAr?$AA?$AA@ ; `string'
PUBLIC	??_C@_1CM@BIEIIFPA@?$AAp?$AAa?$AAr?$AAs?$AAe?$AAr?$AA?5?$AAs?$AAt?$AAa?$AAc?$AAk?$AA?5?$AAo?$AAv?$AAe?$AAr?$AAf?$AAl?$AAo?$AAw?$AA?$AA@ ; `string'
PUBLIC	??_C@_1CG@DJMDIOIE@?$AAP?$AAr?$AAo?$AAl?$AAo?$AAg?$AA?5?$AAp?$AAa?$AAr?$AAs?$AAe?$AA?5?$AAe?$AAr?$AAr?$AAo?$AAr?$AA?$AA@ ; `string'
?yynerrs@@3HA DD 01H DUP (?)				; yynerrs
?yychar@@3HA DD	01H DUP (?)				; yychar
?yylval@@3TYYSTYPE@@A DD 01H DUP (?)			; yylval
;	COMDAT ??_C@_1CG@DJMDIOIE@?$AAP?$AAr?$AAo?$AAl?$AAo?$AAg?$AA?5?$AAp?$AAa?$AAr?$AAs?$AAe?$AA?5?$AAe?$AAr?$AAr?$AAo?$AAr?$AA?$AA@
CONST	SEGMENT
??_C@_1CG@DJMDIOIE@?$AAP?$AAr?$AAo?$AAl?$AAo?$AAg?$AA?5?$AAp?$AAa?$AAr?$AAs?$AAe?$AA?5?$AAe?$AAr?$AAr?$AAo?$AAr?$AA?$AA@ DB 'P'
	DB	00H, 'r', 00H, 'o', 00H, 'l', 00H, 'o', 00H, 'g', 00H, ' ', 00H
	DB	'p', 00H, 'a', 00H, 'r', 00H, 's', 00H, 'e', 00H, ' ', 00H, 'e'
	DB	00H, 'r', 00H, 'r', 00H, 'o', 00H, 'r', 00H, 00H, 00H ; `string'
CONST	ENDS
;	COMDAT ??_C@_1CM@BIEIIFPA@?$AAp?$AAa?$AAr?$AAs?$AAe?$AAr?$AA?5?$AAs?$AAt?$AAa?$AAc?$AAk?$AA?5?$AAo?$AAv?$AAe?$AAr?$AAf?$AAl?$AAo?$AAw?$AA?$AA@
CONST	SEGMENT
??_C@_1CM@BIEIIFPA@?$AAp?$AAa?$AAr?$AAs?$AAe?$AAr?$AA?5?$AAs?$AAt?$AAa?$AAc?$AAk?$AA?5?$AAo?$AAv?$AAe?$AAr?$AAf?$AAl?$AAo?$AAw?$AA?$AA@ DB 'p'
	DB	00H, 'a', 00H, 'r', 00H, 's', 00H, 'e', 00H, 'r', 00H, ' ', 00H
	DB	's', 00H, 't', 00H, 'a', 00H, 'c', 00H, 'k', 00H, ' ', 00H, 'o'
	DB	00H, 'v', 00H, 'e', 00H, 'r', 00H, 'f', 00H, 'l', 00H, 'o', 00H
	DB	'w', 00H, 00H, 00H				; `string'
CONST	ENDS
;	COMDAT ??_C@_1BK@ECDIFIKG@?$AAs?$AAy?$AAn?$AAt?$AAa?$AAx?$AA?5?$AAe?$AAr?$AAr?$AAo?$AAr?$AA?$AA@
CONST	SEGMENT
??_C@_1BK@ECDIFIKG@?$AAs?$AAy?$AAn?$AAt?$AAa?$AAx?$AA?5?$AAe?$AAr?$AAr?$AAo?$AAr?$AA?$AA@ DB 's'
	DB	00H, 'y', 00H, 'n', 00H, 't', 00H, 'a', 00H, 'x', 00H, ' ', 00H
	DB	'e', 00H, 'r', 00H, 'r', 00H, 'o', 00H, 'r', 00H, 00H, 00H ; `string'
_szStringVal DD	FLAT:??_C@_13HADIAKP@?$AAS?$AA?$AA@
_szDwordVal DD	FLAT:??_C@_13MKMNOPIJ@?$AAD?$AA?$AA@
_szBinaryVal DD	FLAT:??_C@_13OPKGLAFF@?$AAB?$AA?$AA@
_szValToken DD	FLAT:??_C@_17LLMMEOJD@?$AAV?$AAa?$AAl?$AA?$AA@
_szForceRemove DD FLAT:??_C@_1BI@JFAIJMHL@?$AAF?$AAo?$AAr?$AAc?$AAe?$AAR?$AAe?$AAm?$AAo?$AAv?$AAe?$AA?$AA@
_szNoRemove DD	FLAT:??_C@_1BC@GCKHIPE@?$AAN?$AAo?$AAR?$AAe?$AAm?$AAo?$AAv?$AAe?$AA?$AA@
_szDelete DD	FLAT:??_C@_1O@JDLOHAN@?$AAD?$AAe?$AAl?$AAe?$AAt?$AAe?$AA?$AA@
_yytranslate DB	00H
	DB	02H
	DB	02H
	DB	02H
	DB	02H
	DB	02H
	DB	02H
	DB	02H
	DB	02H
	DB	02H
	DB	02H
	DB	02H
	DB	02H
	DB	02H
	DB	02H
	DB	02H
	DB	02H
	DB	02H
	DB	02H
	DB	02H
	DB	02H
	DB	02H
	DB	02H
	DB	02H
	DB	02H
	DB	02H
	DB	02H
	DB	02H
	DB	02H
	DB	02H
	DB	02H
	DB	02H
	DB	02H
	DB	02H
	DB	02H
	DB	02H
	DB	02H
	DB	02H
	DB	02H
	DB	02H
	DB	02H
	DB	02H
	DB	02H
	DB	02H
	DB	02H
	DB	02H
	DB	02H
	DB	02H
	DB	02H
	DB	02H
	DB	02H
	DB	02H
	DB	02H
	DB	02H
	DB	02H
	DB	02H
	DB	02H
	DB	02H
	DB	02H
	DB	02H
	DB	02H
	DB	02H
	DB	02H
	DB	02H
	DB	02H
	DB	02H
	DB	02H
	DB	02H
	DB	02H
	DB	02H
	DB	02H
	DB	02H
	DB	02H
	DB	02H
	DB	02H
	DB	02H
	DB	02H
	DB	02H
	DB	02H
	DB	02H
	DB	02H
	DB	02H
	DB	02H
	DB	02H
	DB	02H
	DB	02H
	DB	02H
	DB	02H
	DB	02H
	DB	02H
	DB	02H
	DB	02H
	DB	02H
	DB	02H
	DB	02H
	DB	02H
	DB	02H
	DB	02H
	DB	02H
	DB	02H
	DB	02H
	DB	02H
	DB	02H
	DB	02H
	DB	02H
	DB	02H
	DB	02H
	DB	02H
	DB	02H
	DB	02H
	DB	02H
	DB	02H
	DB	02H
	DB	02H
	DB	02H
	DB	02H
	DB	02H
	DB	02H
	DB	02H
	DB	02H
	DB	02H
	DB	02H
	DB	02H
	DB	02H
	DB	02H
	DB	02H
	DB	02H
	DB	02H
	DB	02H
	DB	02H
	DB	02H
	DB	02H
	DB	02H
	DB	02H
	DB	02H
	DB	02H
	DB	02H
	DB	02H
	DB	02H
	DB	02H
	DB	02H
	DB	02H
	DB	02H
	DB	02H
	DB	02H
	DB	02H
	DB	02H
	DB	02H
	DB	02H
	DB	02H
	DB	02H
	DB	02H
	DB	02H
	DB	02H
	DB	02H
	DB	02H
	DB	02H
	DB	02H
	DB	02H
	DB	02H
	DB	02H
	DB	02H
	DB	02H
	DB	02H
	DB	02H
	DB	02H
	DB	02H
	DB	02H
	DB	02H
	DB	02H
	DB	02H
	DB	02H
	DB	02H
	DB	02H
	DB	02H
	DB	02H
	DB	02H
	DB	02H
	DB	02H
	DB	02H
	DB	02H
	DB	02H
	DB	02H
	DB	02H
	DB	02H
	DB	02H
	DB	02H
	DB	02H
	DB	02H
	DB	02H
	DB	02H
	DB	02H
	DB	02H
	DB	02H
	DB	02H
	DB	02H
	DB	02H
	DB	02H
	DB	02H
	DB	02H
	DB	02H
	DB	02H
	DB	02H
	DB	02H
	DB	02H
	DB	02H
	DB	02H
	DB	02H
	DB	02H
	DB	02H
	DB	02H
	DB	02H
	DB	02H
	DB	02H
	DB	02H
	DB	02H
	DB	02H
	DB	02H
	DB	02H
	DB	02H
	DB	02H
	DB	02H
	DB	02H
	DB	02H
	DB	02H
	DB	02H
	DB	02H
	DB	02H
	DB	02H
	DB	02H
	DB	02H
	DB	02H
	DB	02H
	DB	02H
	DB	02H
	DB	02H
	DB	02H
	DB	02H
	DB	02H
	DB	02H
	DB	02H
	DB	02H
	DB	02H
	DB	02H
	DB	02H
	DB	02H
	DB	02H
	DB	02H
	DB	02H
	DB	02H
	DB	02H
	DB	02H
	DB	02H
	DB	02H
	DB	02H
	DB	02H
	DB	01H
	DB	02H
	DB	03H
	DB	04H
	DB	05H
	DB	06H
	DB	07H
	DB	08H
	DB	09H
	DB	0aH
	DB	0bH
	DB	0cH
	DB	0dH
	DB	0eH
	DB	0fH
	DB	010H
	DB	011H
	DB	012H
	DB	013H
	DB	014H
	DB	015H
	DB	016H
	DB	017H
	DB	018H
	DB	019H
	DB	01aH
	DB	01bH
	DB	01cH
	DB	01dH
	DB	01eH
	DB	01fH
	DB	020H
	DB	021H
	DB	022H
	DB	023H
	DB	024H
	DB	025H
	DB	026H
	DB	027H
	DB	028H
	DB	029H
	DB	02aH
	DB	02bH
	DB	02cH
	DB	02dH
	DB	02eH
	DB	02fH
	DB	030H
	DB	031H
	DB	032H
	DB	033H
	DB	034H
	DB	035H
	DB	036H
	DB	037H
	DB	038H
	DB	039H
	ORG $+7
_yyr1	DB	00H
	DB	03aH
	DB	03bH
	DB	03cH
	DB	03dH
	DB	03dH
	DB	03eH
	DB	03eH
	DB	03fH
	DB	03fH
	DB	03fH
	DB	03fH
	DB	040H
	DB	041H
	DB	042H
	DB	042H
	DB	043H
	DB	044H
	DB	045H
	DB	045H
	DB	046H
	DB	046H
	DB	046H
	DB	047H
	DB	048H
	DB	048H
	DB	049H
	DB	049H
	DB	04aH
	DB	04bH
	DB	04bH
	DB	04bH
	DB	04bH
	DB	04cH
	DB	04dH
	DB	04dH
	DB	04eH
	DB	04eH
	DB	04fH
	DB	04fH
	DB	04fH
	DB	04fH
	DB	04fH
	DB	04fH
	DB	050H
	DB	051H
	DB	051H
	DB	052H
	DB	052H
	DB	053H
	DB	053H
	DB	054H
	DB	054H
	DB	055H
	DB	056H
	DB	057H
	DB	057H
	DB	058H
	DB	058H
	DB	059H
	DB	059H
	DB	05aH
	DB	05aH
	DB	05bH
	DB	05cH
	DB	05dH
	DB	05dH
	DB	05dH
	DB	05dH
	DB	05eH
	DB	05eH
	DB	05fH
	DB	05fH
	DB	05fH
	DB	060H
	DB	061H
	DB	061H
	DB	062H
	DB	063H
	DB	064H
	DB	064H
	DB	065H
	DB	066H
	DB	066H
	DB	067H
	DB	067H
	DB	068H
	DB	069H
	DB	069H
	DB	06aH
	DB	06aH
	DB	06aH
	DB	06bH
	DB	06cH
	DB	06cH
	DB	06dH
	DB	06eH
	DB	06eH
	DB	06eH
	DB	06fH
	DB	070H
	DB	070H
	DB	070H
	DB	070H
	DB	070H
	DB	070H
	DB	070H
	DB	071H
	DB	071H
	DB	072H
	DB	073H
	DB	073H
	DB	074H
	DB	075H
	DB	075H
	DB	076H
	DB	076H
	DB	076H
	DB	077H
	DB	077H
	DB	078H
	DB	079H
	DB	07aH
	DB	07bH
	DB	079H
	DB	079H
	DB	07cH
	DB	07cH
	DB	07dH
	DB	07dH
	DB	07eH
	DB	07eH
	DB	07fH
	DB	080H
	DB	080H
	DB	081H
	DB	082H
	DB	083H
	DB	084H
	DB	085H
	DB	086H
	DB	087H
	DB	088H
	DB	089H
	DB	08aH
	DB	08bH
	DB	08cH
	DB	08dH
	DB	08eH
	ORG $+3
_yyr2	DB	00H
	DB	02H
	DB	02H
	DB	03H
	DB	00H
	DB	01H
	DB	03H
	DB	02H
	DB	02H
	DB	04H
	DB	06H
	DB	04H
	DB	03H
	DB	03H
	DB	01H
	DB	01H
	DB	04H
	DB	03H
	DB	00H
	DB	02H
	DB	01H
	DB	01H
	DB	01H
	DB	04H
	DB	00H
	DB	02H
	DB	00H
	DB	02H
	DB	05H
	DB	00H
	DB	02H
	DB	04H
	DB	02H
	DB	04H
	DB	00H
	DB	02H
	DB	01H
	DB	01H
	DB	01H
	DB	01H
	DB	01H
	DB	01H
	DB	01H
	DB	01H
	DB	01H
	DB	03H
	DB	01H
	DB	01H
	DB	01H
	DB	00H
	DB	02H
	DB	01H
	DB	01H
	DB	06H
	DB	09H
	DB	02H
	DB	02H
	DB	01H
	DB	01H
	DB	03H
	DB	05H
	DB	01H
	DB	02H
	DB	04H
	DB	07H
	DB	01H
	DB	01H
	DB	01H
	DB	01H
	DB	02H
	DB	02H
	DB	02H
	DB	02H
	DB	02H
	DB	07H
	DB	01H
	DB	03H
	DB	03H
	DB	05H
	DB	01H
	DB	03H
	DB	03H
	DB	08H
	DB	05H
	DB	01H
	DB	03H
	DB	03H
	DB	00H
	DB	01H
	DB	01H
	DB	01H
	DB	01H
	DB	06H
	DB	00H
	DB	02H
	DB	06H
	DB	01H
	DB	01H
	DB	01H
	DB	01H
	DB	01H
	DB	01H
	DB	01H
	DB	01H
	DB	01H
	DB	01H
	DB	01H
	DB	01H
	DB	01H
	DB	07H
	DB	01H
	DB	05H
	DB	05H
	DB	01H
	DB	05H
	DB	01H
	DB	01H
	DB	02H
	DB	00H
	DB	02H
	DB	06H
	DB	04H
	DB	00H
	DB	00H
	DB	08H
	DB	04H
	DB	04H
	DB	02H
	DB	00H
	DB	02H
	DB	01H
	DB	01H
	DB	01H
	DB	00H
	DB	01H
	DB	01H
	DB	01H
	DB	01H
	DB	01H
	DB	01H
	DB	01H
	DB	01H
	DB	01H
	DB	01H
	DB	01H
	DB	01H
	DB	01H
	DB	01H
	DB	01H
	ORG $+3
_yydefact DB	04H
	DB	00H
	DB	00H
	DB	00H
	DB	012H
	DB	05H
	DB	031H
	DB	084H
	DB	02eH
	DB	085H
	DB	07H
	DB	00H
	DB	01H
	DB	080H
	DB	012H
	DB	02H
	DB	00H
	DB	00H
	DB	084H
	DB	06H
	DB	00H
	DB	00H
	DB	085H
	DB	00H
	DB	00H
	DB	00H
	DB	00H
	DB	013H
	DB	014H
	DB	03H
	DB	012H
	DB	016H
	DB	015H
	DB	032H
	DB	02fH
	DB	030H
	DB	02dH
	DB	085H
	DB	085H
	DB	085H
	DB	085H
	DB	08H
	DB	086H
	DB	00H
	DB	00H
	DB	082H
	DB	012H
	DB	083H
	DB	081H
	DB	00H
	DB	08fH
	DB	018H
	DB	00H
	DB	00H
	DB	00H
	DB	00H
	DB	00H
	DB	00H
	DB	088H
	DB	010H
	DB	085H
	DB	00H
	DB	089H
	DB	01dH
	DB	00H
	DB	00H
	DB	087H
	DB	0cH
	DB	0eH
	DB	0fH
	DB	0dH
	DB	085H
	DB	09H
	DB	0bH
	DB	011H
	DB	00H
	DB	00H
	DB	00H
	DB	017H
	DB	090H
	DB	019H
	DB	00H
	DB	01cH
	DB	00H
	DB	00H
	DB	01eH
	DB	022H
	DB	020H
	DB	0aH
	DB	00H
	DB	00H
	DB	00H
	DB	00H
	DB	08eH
	DB	00H
	DB	093H
	DB	03bH
	DB	01fH
	DB	00H
	DB	02aH
	DB	00H
	DB	00H
	DB	00H
	DB	085H
	DB	023H
	DB	024H
	DB	025H
	DB	02bH
	DB	028H
	DB	033H
	DB	034H
	DB	026H
	DB	027H
	DB	029H
	DB	02cH
	DB	00H
	DB	00H
	DB	00H
	DB	00H
	DB	00H
	DB	021H
	DB	03cH
	DB	08aH
	DB	00H
	DB	00H
	DB	091H
	DB	00H
	DB	05dH
	DB	08dH
	DB	00H
	DB	00H
	DB	00H
	DB	00H
	DB	085H
	DB	00H
	DB	08bH
	DB	00H
	DB	08cH
	DB	00H
	DB	085H
	DB	085H
	DB	041H
	DB	042H
	DB	085H
	DB	085H
	DB	044H
	DB	057H
	DB	057H
	DB	043H
	DB	05eH
	DB	00H
	DB	00H
	DB	00H
	DB	00H
	DB	00H
	DB	00H
	DB	035H
	DB	038H
	DB	085H
	DB	00H
	DB	03dH
	DB	037H
	DB	00H
	DB	00H
	DB	05aH
	DB	05bH
	DB	059H
	DB	045H
	DB	058H
	DB	046H
	DB	00H
	DB	05cH
	DB	00H
	DB	00H
	DB	078H
	DB	085H
	DB	03aH
	DB	039H
	DB	03eH
	DB	00H
	DB	085H
	DB	085H
	DB	085H
	DB	057H
	DB	057H
	DB	057H
	DB	040H
	DB	00H
	DB	085H
	DB	085H
	DB	00H
	DB	00H
	DB	00H
	DB	00H
	DB	00H
	DB	04fH
	DB	048H
	DB	049H
	DB	047H
	DB	085H
	DB	00H
	DB	067H
	DB	068H
	DB	069H
	DB	063H
	DB	06aH
	DB	064H
	DB	065H
	DB	066H
	DB	00H
	DB	060H
	DB	061H
	DB	062H
	DB	06bH
	DB	06cH
	DB	07aH
	DB	07dH
	DB	079H
	DB	036H
	DB	03fH
	DB	053H
	DB	085H
	DB	085H
	DB	054H
	DB	04eH
	DB	085H
	DB	085H
	DB	085H
	DB	085H
	DB	04bH
	DB	00H
	DB	00H
	DB	076H
	DB	00H
	DB	00H
	DB	00H
	DB	00H
	DB	050H
	DB	00H
	DB	00H
	DB	092H
	DB	085H
	DB	071H
	DB	085H
	DB	00H
	DB	073H
	DB	074H
	DB	05fH
	DB	00H
	DB	07bH
	DB	056H
	DB	00H
	DB	055H
	DB	051H
	DB	04dH
	DB	04aH
	DB	04cH
	DB	00H
	DB	00H
	DB	077H
	DB	094H
	DB	075H
	DB	085H
	DB	052H
	DB	070H
	DB	085H
	DB	085H
	DB	06eH
	DB	07cH
	DB	00H
	DB	00H
	DB	072H
	DB	06dH
	DB	085H
	DB	00H
	DB	06fH
_yydefgoto DW	0ffffH
	DW	02H
	DW	03H
	DW	04H
	DW	05H
	DW	013H
	DW	027H
	DW	028H
	DW	046H
	DW	09H
	DW	02bH
	DW	010H
	DW	01bH
	DW	01cH
	DW	040H
	DW	01dH
	DW	01eH
	DW	04bH
	DW	057H
	DW	05cH
	DW	068H
	DW	069H
	DW	06aH
	DW	01fH
	DW	024H
	DW	011H
	DW	06cH
	DW	06dH
	DW	06eH
	DW	08aH
	DW	0afH
	DW	055H
	DW	09dH
	DW	09eH
	DW	06fH
	DW	090H
	DW	091H
	DW	0b6H
	DW	0b7H
	DW	0e4H
	DW	0e5H
	DW	0b8H
	DW	0c2H
	DW	0e2H
	DW	094H
	DW	0deH
	DW	0dfH
	DW	0a7H
	DW	0a8H
	DW	070H
	DW	085H
	DW	095H
	DW	0d1H
	DW	0d2H
	DW	0d3H
	DW	0d4H
	DW	0d5H
	DW	010aH
	DW	0d6H
	DW	0f1H
	DW	0f7H
	DW	0f8H
	DW	071H
	DW	09aH
	DW	0e9H
	DW	0106H
	DW	0fH
	DW	017H
	DW	030H
	DW	020H
	DW	02cH
	DW	043H
	DW	03bH
	DW	03fH
	DW	07cH
	DW	088H
	DW	08cH
	DW	081H
	DW	05eH
	DW	033H
	DW	050H
	DW	0b9H
	DW	0f2H
	DW	060H
	DW	0105H
	ORG $+6
_yypact	DW	0dH
	DW	01H
	DW	035H
	DW	014H
	DW	0ff20H
	DW	0ff20H
	DW	0ff20H
	DW	0ff20H
	DW	0ff20H
	DW	034H
	DW	0ff20H
	DW	021H
	DW	0ff20H
	DW	0ff20H
	DW	0ff20H
	DW	0ff20H
	DW	050H
	DW	09H
	DW	02cH
	DW	0ff20H
	DW	066H
	DW	033H
	DW	040H
	DW	01cH
	DW	03H
	DW	04cH
	DW	05fH
	DW	0ff20H
	DW	0ff20H
	DW	0ff20H
	DW	0ff20H
	DW	0ff20H
	DW	0ff20H
	DW	0ff20H
	DW	0ff20H
	DW	0ff20H
	DW	0ff20H
	DW	040H
	DW	040H
	DW	034H
	DW	040H
	DW	0ff20H
	DW	0ff20H
	DW	072H
	DW	04dH
	DW	0ff20H
	DW	0ff20H
	DW	0ff20H
	DW	0ff20H
	DW	078H
	DW	0ff20H
	DW	04cH
	DW	05eH
	DW	07bH
	DW	067H
	DW	070H
	DW	079H
	DW	07eH
	DW	0ff20H
	DW	0ff20H
	DW	040H
	DW	07H
	DW	0ff20H
	DW	02dH
	DW	080H
	DW	082H
	DW	0ff20H
	DW	0ff20H
	DW	0ff20H
	DW	0ff20H
	DW	0ff20H
	DW	040H
	DW	0ff20H
	DW	0ff20H
	DW	0ff20H
	DW	086H
	DW	065H
	DW	07aH
	DW	0ff20H
	DW	0ff20H
	DW	0ff20H
	DW	087H
	DW	0ff20H
	DW	04cH
	DW	04cH
	DW	031H
	DW	0ff20H
	DW	0ff20H
	DW	0ff20H
	DW	08dH
	DW	092H
	DW	07aH
	DW	017H
	DW	0ff20H
	DW	04cH
	DW	0ff20H
	DW	0ff20H
	DW	0ff20H
	DW	04cH
	DW	0ff20H
	DW	04cH
	DW	04cH
	DW	04cH
	DW	040H
	DW	0ff20H
	DW	0ff20H
	DW	0ff20H
	DW	0ff20H
	DW	0ff20H
	DW	0ff20H
	DW	0ff20H
	DW	0ff20H
	DW	0ff20H
	DW	0ff20H
	DW	0ff20H
	DW	092H
	DW	011H
	DW	0a0H
	DW	0a0H
	DW	0a1H
	DW	0ff20H
	DW	0ff20H
	DW	0ff20H
	DW	04cH
	DW	04cH
	DW	0ff20H
	DW	04cH
	DW	0ff20H
	DW	0ff20H
	DW	04cH
	DW	0a2H
	DW	0fffaH
	DW	052H
	DW	034H
	DW	06bH
	DW	0ff20H
	DW	04cH
	DW	0ff20H
	DW	094H
	DW	034H
	DW	040H
	DW	0ff20H
	DW	0ff20H
	DW	040H
	DW	040H
	DW	0ff20H
	DW	047H
	DW	047H
	DW	0ff20H
	DW	0ff20H
	DW	0a0H
	DW	095H
	DW	04cH
	DW	04cH
	DW	096H
	DW	0fffaH
	DW	0ff20H
	DW	0ff20H
	DW	040H
	DW	091H
	DW	0ff20H
	DW	0ff20H
	DW	025H
	DW	097H
	DW	0ff20H
	DW	0ff20H
	DW	0ff20H
	DW	0ff20H
	DW	0ff20H
	DW	0ff20H
	DW	04cH
	DW	0ff20H
	DW	09fH
	DW	0a3H
	DW	0ff20H
	DW	040H
	DW	0ff20H
	DW	0ff20H
	DW	0ff20H
	DW	04cH
	DW	040H
	DW	040H
	DW	040H
	DW	047H
	DW	047H
	DW	047H
	DW	0ff20H
	DW	0deH
	DW	034H
	DW	040H
	DW	09dH
	DW	0a0H
	DW	02fH
	DW	0eH
	DW	01dH
	DW	08cH
	DW	0ff20H
	DW	0ff20H
	DW	0ff20H
	DW	040H
	DW	04cH
	DW	0ff20H
	DW	0ff20H
	DW	0ff20H
	DW	0ff20H
	DW	0ff20H
	DW	0ff20H
	DW	0ff20H
	DW	0ff20H
	DW	04cH
	DW	0ff20H
	DW	0ff20H
	DW	0ff20H
	DW	0ff20H
	DW	0ff20H
	DW	0ff20H
	DW	0ff20H
	DW	0ff20H
	DW	0ff20H
	DW	0ff20H
	DW	0ff20H
	DW	040H
	DW	040H
	DW	0ff20H
	DW	0ff20H
	DW	040H
	DW	040H
	DW	040H
	DW	040H
	DW	0ff20H
	DW	0aaH
	DW	093H
	DW	0ffdfH
	DW	0abH
	DW	0a0H
	DW	032H
	DW	0eH
	DW	0ff20H
	DW	0eH
	DW	03cH
	DW	0ff20H
	DW	040H
	DW	0ff20H
	DW	040H
	DW	04cH
	DW	0ff20H
	DW	0ff20H
	DW	0ff20H
	DW	0b6H
	DW	0ff20H
	DW	0ff20H
	DW	098H
	DW	0ff20H
	DW	0ff20H
	DW	0ff20H
	DW	0ff20H
	DW	0ff20H
	DW	041H
	DW	0a0H
	DW	0ff20H
	DW	0ff20H
	DW	0ff20H
	DW	040H
	DW	0ff20H
	DW	0ff20H
	DW	040H
	DW	040H
	DW	0ff20H
	DW	0ff20H
	DW	0aaH
	DW	043H
	DW	0ff20H
	DW	0ff20H
	DW	040H
	DW	0a0H
	DW	0ff20H
_yypgoto DW	0ff20H
	DW	0ff20H
	DW	0ff20H
	DW	0ff20H
	DW	0ff20H
	DW	0ff20H
	DW	0ff20H
	DW	08aH
	DW	0ff20H
	DW	0ff20H
	DW	06aH
	DW	029H
	DW	0a6H
	DW	0ff20H
	DW	0ff20H
	DW	0ff20H
	DW	0ff20H
	DW	0ff20H
	DW	068H
	DW	0ff20H
	DW	0ff20H
	DW	0ff20H
	DW	0ff20H
	DW	00H
	DW	0ff20H
	DW	0ff20H
	DW	0ff20H
	DW	0ff20H
	DW	0ff20H
	DW	0ff20H
	DW	0ff20H
	DW	0ff9dH
	DW	0ff20H
	DW	0ff20H
	DW	0ff20H
	DW	0ff20H
	DW	0ff20H
	DW	0ff21H
	DW	042H
	DW	0ff20H
	DW	0ffd5H
	DW	044H
	DW	0ff20H
	DW	0ff20H
	DW	0ff20H
	DW	0ff20H
	DW	0ffdcH
	DW	0ff76H
	DW	0ff20H
	DW	0ff20H
	DW	0ff20H
	DW	0ff20H
	DW	0ff20H
	DW	0ff20H
	DW	0ff20H
	DW	0ff20H
	DW	0ff20H
	DW	0ff20H
	DW	0ff20H
	DW	0ff20H
	DW	0ff20H
	DW	0ff20H
	DW	0ff20H
	DW	0ff20H
	DW	0ff20H
	DW	0ff20H
	DW	0ff20H
	DW	0ff20H
	DW	0ff20H
	DW	03aH
	DW	0fff7H
	DW	0ff20H
	DW	0ff20H
	DW	0ff20H
	DW	0ff20H
	DW	0ff20H
	DW	02eH
	DW	0ff20H
	DW	0ff20H
	DW	0ff20H
	DW	0ff20H
	DW	0ff90H
	DW	0ffbdH
	DW	058H
	DW	0ff20H
	ORG $+6
_yytable DW	015H
	DW	0aH
	DW	06H
	DW	0ff81H
	DW	06H
	DW	07eH
	DW	07fH
	DW	0ff82H
	DW	06H
	DW	0a9H
	DW	021H
	DW	089H
	DW	0f4H
	DW	0fdH
	DW	01aH
	DW	0feH
	DW	0f5H
	DW	07dH
	DW	01aH
	DW	0f6H
	DW	07aH
	DW	07H
	DW	01H
	DW	07H
	DW	06H
	DW	053H
	DW	054H
	DW	07H
	DW	022H
	DW	06H
	DW	038H
	DW	039H
	DW	08bH
	DW	062H
	DW	063H
	DW	064H
	DW	065H
	DW	066H
	DW	0aaH
	DW	01aH
	DW	07dH
	DW	0dH
	DW	0eH
	DW	07H
	DW	07bH
	DW	0c4H
	DW	0c5H
	DW	0c6H
	DW	07H
	DW	02dH
	DW	02eH
	DW	04aH
	DW	0b5H
	DW	0cH
	DW	04dH
	DW	018H
	DW	0b0H
	DW	067H
	DW	08H
	DW	0bH
	DW	08H
	DW	016H
	DW	051H
	DW	0ff7aH
	DW	08H
	DW	012H
	DW	023H
	DW	014H
	DW	0e0H
	DW	02aH
	DW	029H
	DW	034H
	DW	012H
	DW	0e1H
	DW	0b4H
	DW	0b5H
	DW	05bH
	DW	0ff7aH
	DW	0ff7bH
	DW	0dbH
	DW	08H
	DW	06H
	DW	0ff7bH
	DW	031H
	DW	02aH
	DW	08H
	DW	0dcH
	DW	03dH
	DW	019H
	DW	0fbH
	DW	0ddH
	DW	01aH
	DW	06bH
	DW	0ddH
	DW	078H
	DW	06H
	DW	07H
	DW	037H
	DW	032H
	DW	0ffH
	DW	07H
	DW	0ffe6H
	DW	0ffe6H
	DW	0e3H
	DW	0108H
	DW	01aH
	DW	0110H
	DW	03cH
	DW	0109H
	DW	041H
	DW	0111H
	DW	0a4H
	DW	0a5H
	DW	0a6H
	DW	07H
	DW	0ffe5H
	DW	0ffe5H
	DW	08dH
	DW	08eH
	DW	03aH
	DW	08fH
	DW	04cH
	DW	0faH
	DW	03eH
	DW	097H
	DW	025H
	DW	026H
	DW	042H
	DW	044H
	DW	045H
	DW	0a0H
	DW	0a1H
	DW	053H
	DW	054H
	DW	0a2H
	DW	0a3H
	DW	026H
	DW	08H
	DW	098H
	DW	099H
	DW	048H
	DW	059H
	DW	05aH
	DW	035H
	DW	036H
	DW	049H
	DW	010bH
	DW	04eH
	DW	04fH
	DW	0b2H
	DW	072H
	DW	08H
	DW	073H
	DW	052H
	DW	058H
	DW	056H
	DW	074H
	DW	05dH
	DW	075H
	DW	076H
	DW	077H
	DW	05fH
	DW	0113H
	DW	07dH
	DW	080H
	DW	087H
	DW	0beH
	DW	09cH
	DW	0abH
	DW	0aeH
	DW	0baH
	DW	0c0H
	DW	0c1H
	DW	0c3H
	DW	0b3H
	DW	0bcH
	DW	0daH
	DW	0f0H
	DW	0bdH
	DW	0d8H
	DW	0d9H
	DW	082H
	DW	083H
	DW	0e3H
	DW	084H
	DW	0f3H
	DW	0f9H
	DW	086H
	DW	0104H
	DW	02fH
	DW	0e6H
	DW	096H
	DW	0107H
	DW	047H
	DW	09bH
	DW	061H
	DW	0100H
	DW	09fH
	DW	092H
	DW	0fcH
	DW	093H
	DW	0b1H
	DW	010fH
	DW	079H
	DW	00H
	DW	00H
	DW	00H
	DW	00H
	DW	00H
	DW	00H
	DW	0acH
	DW	0adH
	DW	0eaH
	DW	0ebH
	DW	00H
	DW	00H
	DW	0ecH
	DW	0edH
	DW	0eeH
	DW	0efH
	DW	00H
	DW	00H
	DW	00H
	DW	00H
	DW	00H
	DW	00H
	DW	00H
	DW	00H
	DW	0bbH
	DW	00H
	DW	00H
	DW	00H
	DW	0101H
	DW	00H
	DW	0102H
	DW	00H
	DW	00H
	DW	0bfH
	DW	00H
	DW	00H
	DW	00H
	DW	00H
	DW	00H
	DW	00H
	DW	00H
	DW	00H
	DW	0d7H
	DW	00H
	DW	00H
	DW	00H
	DW	00H
	DW	00H
	DW	00H
	DW	010cH
	DW	00H
	DW	00H
	DW	010dH
	DW	010eH
	DW	0e7H
	DW	00H
	DW	0c7H
	DW	00H
	DW	00H
	DW	00H
	DW	0112H
	DW	00H
	DW	00H
	DW	0e8H
	DW	0c8H
	DW	0c9H
	DW	0caH
	DW	00H
	DW	0cbH
	DW	0ccH
	DW	00H
	DW	0cdH
	DW	0ceH
	DW	0cfH
	DW	0d0H
	DW	00H
	DW	00H
	DW	00H
	DW	00H
	DW	00H
	DW	00H
	DW	00H
	DW	00H
	DW	00H
	DW	00H
	DW	00H
	DW	00H
	DW	00H
	DW	00H
	DW	00H
	DW	00H
	DW	00H
	DW	00H
	DW	00H
	DW	00H
	DW	00H
	DW	00H
	DW	00H
	DW	0103H
	ORG $+2
_yycheck DW	09H
	DW	01H
	DW	01H
	DW	00H
	DW	01H
	DW	075H
	DW	076H
	DW	00H
	DW	01H
	DW	093H
	DW	01H
	DW	011H
	DW	02dH
	DW	0ecH
	DW	0bH
	DW	0eeH
	DW	031H
	DW	03H
	DW	0bH
	DW	034H
	DW	03H
	DW	014H
	DW	09H
	DW	014H
	DW	01H
	DW	01fH
	DW	020H
	DW	014H
	DW	013H
	DW	01H
	DW	027H
	DW	028H
	DW	083H
	DW	0aH
	DW	0bH
	DW	0cH
	DW	0dH
	DW	0eH
	DW	096H
	DW	0bH
	DW	03H
	DW	015H
	DW	016H
	DW	014H
	DW	01bH
	DW	0b7H
	DW	0b8H
	DW	0b9H
	DW	014H
	DW	015H
	DW	016H
	DW	03cH
	DW	026H
	DW	00H
	DW	03fH
	DW	0eH
	DW	09bH
	DW	022H
	DW	039H
	DW	01H
	DW	039H
	DW	01cH
	DW	047H
	DW	013H
	DW	039H
	DW	014H
	DW	039H
	DW	09H
	DW	027H
	DW	014H
	DW	013H
	DW	01eH
	DW	014H
	DW	02cH
	DW	025H
	DW	026H
	DW	055H
	DW	021H
	DW	021H
	DW	0bfH
	DW	039H
	DW	01H
	DW	021H
	DW	019H
	DW	014H
	DW	039H
	DW	027H
	DW	02eH
	DW	08H
	DW	027H
	DW	02bH
	DW	0bH
	DW	05cH
	DW	02bH
	DW	067H
	DW	01H
	DW	014H
	DW	027H
	DW	03H
	DW	027H
	DW	014H
	DW	015H
	DW	016H
	DW	02bH
	DW	027H
	DW	0bH
	DW	027H
	DW	01eH
	DW	02bH
	DW	033H
	DW	02bH
	DW	028H
	DW	029H
	DW	02aH
	DW	014H
	DW	015H
	DW	016H
	DW	023H
	DW	024H
	DW	05H
	DW	026H
	DW	03fH
	DW	0eaH
	DW	03H
	DW	085H
	DW	017H
	DW	018H
	DW	04H
	DW	019H
	DW	01aH
	DW	08bH
	DW	08cH
	DW	01fH
	DW	020H
	DW	08fH
	DW	090H
	DW	018H
	DW	039H
	DW	01fH
	DW	020H
	DW	013H
	DW	053H
	DW	054H
	DW	025H
	DW	026H
	DW	013H
	DW	0102H
	DW	013H
	DW	012H
	DW	09eH
	DW	05cH
	DW	039H
	DW	05eH
	DW	013H
	DW	013H
	DW	021H
	DW	062H
	DW	010H
	DW	064H
	DW	065H
	DW	066H
	DW	0fH
	DW	0112H
	DW	03H
	DW	03H
	DW	03H
	DW	0afH
	DW	013H
	DW	013H
	DW	013H
	DW	013H
	DW	0b4H
	DW	0b5H
	DW	0b6H
	DW	01dH
	DW	010H
	DW	013H
	DW	07H
	DW	0fH
	DW	0bcH
	DW	0bdH
	DW	07bH
	DW	07cH
	DW	02bH
	DW	07eH
	DW	026H
	DW	0fH
	DW	081H
	DW	06H
	DW	017H
	DW	0c7H
	DW	085H
	DW	028H
	DW	037H
	DW	088H
	DW	05bH
	DW	0efH
	DW	08bH
	DW	084H
	DW	0ebH
	DW	084H
	DW	09bH
	DW	010dH
	DW	073H
	DW	0ffffH
	DW	0ffffH
	DW	0ffffH
	DW	0ffffH
	DW	0ffffH
	DW	0ffffH
	DW	098H
	DW	099H
	DW	0ddH
	DW	0deH
	DW	0ffffH
	DW	0ffffH
	DW	0e1H
	DW	0e2H
	DW	0e3H
	DW	0e4H
	DW	0ffffH
	DW	0ffffH
	DW	0ffffH
	DW	0ffffH
	DW	0ffffH
	DW	0ffffH
	DW	0ffffH
	DW	0ffffH
	DW	0aaH
	DW	0ffffH
	DW	0ffffH
	DW	0ffffH
	DW	0f1H
	DW	0ffffH
	DW	0f3H
	DW	0ffffH
	DW	0ffffH
	DW	0b3H
	DW	0ffffH
	DW	0ffffH
	DW	0ffffH
	DW	0ffffH
	DW	0ffffH
	DW	0ffffH
	DW	0ffffH
	DW	0ffffH
	DW	0bcH
	DW	0ffffH
	DW	0ffffH
	DW	0ffffH
	DW	0ffffH
	DW	0ffffH
	DW	0ffffH
	DW	0106H
	DW	0ffffH
	DW	0ffffH
	DW	0109H
	DW	010aH
	DW	0c8H
	DW	0ffffH
	DW	026H
	DW	0ffffH
	DW	0ffffH
	DW	0ffffH
	DW	0111H
	DW	0ffffH
	DW	0ffffH
	DW	0d1H
	DW	02eH
	DW	02fH
	DW	030H
	DW	0ffffH
	DW	032H
	DW	033H
	DW	0ffffH
	DW	035H
	DW	036H
	DW	037H
	DW	038H
	DW	0ffffH
	DW	0ffffH
	DW	0ffffH
	DW	0ffffH
	DW	0ffffH
	DW	0ffffH
	DW	0ffffH
	DW	0ffffH
	DW	0ffffH
	DW	0ffffH
	DW	0ffffH
	DW	0ffffH
	DW	0ffffH
	DW	0ffffH
	DW	0ffffH
	DW	0ffffH
	DW	0ffffH
	DW	0ffffH
	DW	0ffffH
	DW	0ffffH
	DW	0ffffH
	DW	0ffffH
	DW	0ffffH
	DW	0f4H
	ORG $+2
_yystos	DB	00H
	DB	09H
	DB	03bH
	DB	03cH
	DB	03dH
	DB	03eH
	DB	01H
	DB	014H
	DB	039H
	DB	043H
	DB	051H
	DB	07fH
	DB	00H
	DB	015H
	DB	016H
	DB	07cH
	DB	045H
	DB	053H
	DB	014H
	DB	03fH
	DB	07fH
	DB	080H
	DB	01cH
	DB	07dH
	DB	045H
	DB	08H
	DB	0bH
	DB	046H
	DB	047H
	DB	049H
	DB	04aH
	DB	051H
	DB	07fH
	DB	01H
	DB	013H
	DB	039H
	DB	052H
	DB	017H
	DB	018H
	DB	040H
	DB	041H
	DB	013H
	DB	014H
	DB	044H
	DB	080H
	DB	015H
	DB	016H
	DB	046H
	DB	07eH
	DB	07fH
	DB	03H
	DB	089H
	DB	045H
	DB	044H
	DB	044H
	DB	07fH
	DB	080H
	DB	080H
	DB	05H
	DB	082H
	DB	01eH
	DB	045H
	DB	03H
	DB	083H
	DB	048H
	DB	07fH
	DB	04H
	DB	081H
	DB	019H
	DB	01aH
	DB	042H
	DB	041H
	DB	013H
	DB	013H
	DB	080H
	DB	04bH
	DB	07fH
	DB	080H
	DB	013H
	DB	012H
	DB	08aH
	DB	080H
	DB	013H
	DB	01fH
	DB	020H
	DB	059H
	DB	021H
	DB	04cH
	DB	013H
	DB	07fH
	DB	07fH
	DB	080H
	DB	04dH
	DB	010H
	DB	088H
	DB	0fH
	DB	08dH
	DB	04cH
	DB	0aH
	DB	0bH
	DB	0cH
	DB	0dH
	DB	0eH
	DB	022H
	DB	04eH
	DB	04fH
	DB	050H
	DB	051H
	DB	054H
	DB	055H
	DB	056H
	DB	05cH
	DB	06bH
	DB	078H
	DB	07fH
	DB	07fH
	DB	07fH
	DB	07fH
	DB	07fH
	DB	07fH
	DB	080H
	DB	08dH
	DB	03H
	DB	01bH
	DB	084H
	DB	03H
	DB	08bH
	DB	08bH
	DB	03H
	DB	087H
	DB	07fH
	DB	07fH
	DB	07fH
	DB	06cH
	DB	07fH
	DB	03H
	DB	085H
	DB	011H
	DB	057H
	DB	059H
	DB	086H
	DB	023H
	DB	024H
	DB	026H
	DB	05dH
	DB	05eH
	DB	060H
	DB	063H
	DB	066H
	DB	06dH
	DB	07fH
	DB	080H
	DB	01fH
	DB	020H
	DB	079H
	DB	07fH
	DB	013H
	DB	05aH
	DB	05bH
	DB	07fH
	DB	080H
	DB	080H
	DB	080H
	DB	080H
	DB	028H
	DB	029H
	DB	02aH
	DB	069H
	DB	06aH
	DB	069H
	DB	08bH
	DB	013H
	DB	07fH
	DB	07fH
	DB	013H
	DB	058H
	DB	059H
	DB	086H
	DB	080H
	DB	01dH
	DB	025H
	DB	026H
	DB	05fH
	DB	060H
	DB	063H
	DB	08bH
	DB	013H
	DB	07fH
	DB	010H
	DB	0fH
	DB	080H
	DB	07fH
	DB	080H
	DB	080H
	DB	064H
	DB	080H
	DB	069H
	DB	069H
	DB	069H
	DB	026H
	DB	02eH
	DB	02fH
	DB	030H
	DB	032H
	DB	033H
	DB	035H
	DB	036H
	DB	037H
	DB	038H
	DB	06eH
	DB	06fH
	DB	070H
	DB	071H
	DB	072H
	DB	074H
	DB	07fH
	DB	080H
	DB	080H
	DB	013H
	DB	08bH
	DB	027H
	DB	02bH
	DB	067H
	DB	068H
	DB	027H
	DB	02cH
	DB	065H
	DB	02bH
	DB	061H
	DB	062H
	DB	080H
	DB	07fH
	DB	07fH
	DB	07aH
	DB	080H
	DB	080H
	DB	080H
	DB	080H
	DB	080H
	DB	080H
	DB	07H
	DB	075H
	DB	08cH
	DB	026H
	DB	02dH
	DB	031H
	DB	034H
	DB	076H
	DB	077H
	DB	0fH
	DB	08bH
	DB	027H
	DB	068H
	DB	05fH
	DB	05fH
	DB	027H
	DB	062H
	DB	080H
	DB	080H
	DB	07fH
	DB	06H
	DB	08eH
	DB	07bH
	DB	028H
	DB	027H
	DB	02bH
	DB	073H
	DB	08bH
	DB	080H
	DB	080H
	DB	080H
	DB	08cH
	DB	027H
	DB	02bH
	DB	080H
	DB	08bH
__bad_alloc_Message DD FLAT:??_C@_0P@GHFPNOJB@bad?5allocation?$AA@
; Function compile flags: /Odtp
; File c:\develop\dscaler423a\dscaler\xml_prolog.tab.cpp
;	COMDAT ?yydestruct@@YAXHPATYYSTYPE@@@Z
_TEXT	SEGMENT
_yytype$ = 8						; size = 4
_yyvaluep$ = 12						; size = 4
?yydestruct@@YAXHPATYYSTYPE@@@Z PROC			; yydestruct, COMDAT

; 1074 : {

  00000	55		 push	 ebp
  00001	8b ec		 mov	 ebp, esp

; 1075 :   /* Pacify ``unused variable'' warnings.  */
; 1076 :   (void) yyvaluep;
; 1077 :   (void) yytype;
; 1078 : }

  00003	5d		 pop	 ebp
  00004	c3		 ret	 0
?yydestruct@@YAXHPATYYSTYPE@@@Z ENDP			; yydestruct
PUBLIC	?yyerror@@YAXPB_W@Z				; yyerror
; Function compile flags: /Odtp
;	COMDAT ?yyerror@@YAXPB_W@Z
_TEXT	SEGMENT
_p_msg$ = 8						; size = 4
?yyerror@@YAXPB_W@Z PROC				; yyerror, COMDAT

; 1707 : {

  00000	55		 push	 ebp
  00001	8b ec		 mov	 ebp, esp

; 1708 :    Xmltv_SyntaxError(_T("Prolog parse error"), p_msg);

  00003	8b 45 08	 mov	 eax, DWORD PTR _p_msg$[ebp]
  00006	50		 push	 eax
  00007	68 00 00 00 00	 push	 OFFSET ??_C@_1CG@DJMDIOIE@?$AAP?$AAr?$AAo?$AAl?$AAo?$AAg?$AA?5?$AAp?$AAa?$AAr?$AAs?$AAe?$AA?5?$AAe?$AAr?$AAr?$AAo?$AAr?$AA?$AA@
  0000c	e8 00 00 00 00	 call	 ?Xmltv_SyntaxError@@YAXPB_W0@Z ; Xmltv_SyntaxError
  00011	83 c4 08	 add	 esp, 8

; 1709 : }

  00014	5d		 pop	 ebp
  00015	c3		 ret	 0
?yyerror@@YAXPB_W@Z ENDP				; yyerror
PUBLIC	__$ArrayPad$
PUBLIC	?yyparse@@YAHXZ					; yyparse
EXTRN	__alloca_probe_16:PROC
; Function compile flags: /Odtp
;	COMDAT ?yyparse@@YAHXZ
_TEXT	SEGMENT
tv191 = -1292						; size = 4
tv162 = -1288						; size = 4
tv79 = -1284						; size = 4
_yyi$138222 = -1280					; size = 4
_yynewbytes$138218 = -1276				; size = 4
_yyi$138210 = -1272					; size = 4
_yynewbytes$138206 = -1268				; size = 4
_yyptr$138196 = -1264					; size = 4
_yyss1$138195 = -1260					; size = 4
_yysize$138190 = -1256					; size = 4
_yyerrstatus$ = -1252					; size = 4
_yyn$ = -1248						; size = 4
_yyresult$ = -1244					; size = 4
_yystate$ = -1240					; size = 4
_yyssp$ = -1236						; size = 4
_yyssa$ = -1232						; size = 400
__$ArrayPad$ = -832					; size = 4
_yyvs$ = -828						; size = 4
_yyss$ = -824						; size = 4
_yyval$ = -820						; size = 4
_yylen$ = -816						; size = 4
_yytoken$ = -812					; size = 4
_yyvsa$ = -808						; size = 800
_yyvsp$ = -8						; size = 4
_yystacksize$ = -4					; size = 4
?yyparse@@YAHXZ PROC					; yyparse, COMDAT

; 1131 : {

  00000	55		 push	 ebp
  00001	8b ec		 mov	 ebp, esp
  00003	81 ec 0c 05 00
	00		 sub	 esp, 1292		; 0000050cH
  00009	a1 00 00 00 00	 mov	 eax, DWORD PTR ___security_cookie
  0000e	33 c5		 xor	 eax, ebp
  00010	89 85 c0 fc ff
	ff		 mov	 DWORD PTR __$ArrayPad$[ebp], eax
  00016	56		 push	 esi

; 1132 : 
; 1133 :   register int yystate;
; 1134 :   register int yyn;
; 1135 :   int yyresult;
; 1136 :   /* Number of tokens to shift before error messages enabled.  */
; 1137 :   int yyerrstatus;
; 1138 :   /* Lookahead token as an internal (translated) token number.  */
; 1139 :   int yytoken = 0;

  00017	c7 85 d4 fc ff
	ff 00 00 00 00	 mov	 DWORD PTR _yytoken$[ebp], 0

; 1140 : 
; 1141 :   /* Three stacks and their tools:
; 1142 :      `yyss': related to states,
; 1143 :      `yyvs': related to semantic values,
; 1144 :      `yyls': related to locations.
; 1145 : 
; 1146 :      Refer to the stacks thru separate pointers, to allow yyoverflow
; 1147 :      to reallocate them elsewhere.  */
; 1148 : 
; 1149 :   /* The state stack.  */
; 1150 :   short    yyssa[YYINITDEPTH];
; 1151 :   short *yyss = yyssa;

  00021	8d 85 30 fb ff
	ff		 lea	 eax, DWORD PTR _yyssa$[ebp]
  00027	89 85 c8 fc ff
	ff		 mov	 DWORD PTR _yyss$[ebp], eax

; 1152 :   register short *yyssp;
; 1153 : 
; 1154 :   /* The semantic value stack.  */
; 1155 :   YYSTYPE yyvsa[YYINITDEPTH];
; 1156 :   YYSTYPE *yyvs = yyvsa;

  0002d	8d 8d d8 fc ff
	ff		 lea	 ecx, DWORD PTR _yyvsa$[ebp]
  00033	89 8d c4 fc ff
	ff		 mov	 DWORD PTR _yyvs$[ebp], ecx

; 1157 :   register YYSTYPE *yyvsp;
; 1158 : 
; 1159 : 
; 1160 : 
; 1161 : #define YYPOPSTACK   (yyvsp--, yyssp--)
; 1162 : 
; 1163 :   YYSIZE_T yystacksize = YYINITDEPTH;

  00039	c7 45 fc c8 00
	00 00		 mov	 DWORD PTR _yystacksize$[ebp], 200 ; 000000c8H

; 1164 : 
; 1165 :   /* The variables used to return semantic value and location from the
; 1166 :      action routines.  */
; 1167 :   YYSTYPE yyval;
; 1168 : 
; 1169 : 
; 1170 :   /* When reducing, the number of symbols on the RHS of the reduced
; 1171 :      rule.  */
; 1172 :   int yylen;
; 1173 : 
; 1174 :   YYDPRINTF ((stderr, _T("Starting parse\n")));
; 1175 : 
; 1176 :   yystate = 0;

  00040	c7 85 28 fb ff
	ff 00 00 00 00	 mov	 DWORD PTR _yystate$[ebp], 0

; 1177 :   yyerrstatus = 0;

  0004a	c7 85 1c fb ff
	ff 00 00 00 00	 mov	 DWORD PTR _yyerrstatus$[ebp], 0

; 1178 :   yynerrs = 0;

  00054	c7 05 00 00 00
	00 00 00 00 00	 mov	 DWORD PTR ?yynerrs@@3HA, 0 ; yynerrs

; 1179 :   yychar = YYEMPTY;        /* Cause a token to be read.  */

  0005e	c7 05 00 00 00
	00 fe ff ff ff	 mov	 DWORD PTR ?yychar@@3HA, -2 ; yychar, fffffffeH

; 1180 : 
; 1181 :   /* Initialize stack pointers.
; 1182 :      Waste one element of value and location stack
; 1183 :      so that they stay on the same level as the state stack.
; 1184 :      The wasted elements are never initialized.  */
; 1185 : 
; 1186 :   yyssp = yyss;

  00068	8b 95 c8 fc ff
	ff		 mov	 edx, DWORD PTR _yyss$[ebp]
  0006e	89 95 2c fb ff
	ff		 mov	 DWORD PTR _yyssp$[ebp], edx

; 1187 :   yyvsp = yyvs;

  00074	8b 85 c4 fc ff
	ff		 mov	 eax, DWORD PTR _yyvs$[ebp]
  0007a	89 45 f8	 mov	 DWORD PTR _yyvsp$[ebp], eax
  0007d	eb 11		 jmp	 SHORT $yysetstate$138186

; 1188 : 
; 1189 :   goto yysetstate;

  0007f	eb 0f		 jmp	 SHORT $yysetstate$138186
$yynewstate$138188:

; 1190 : 
; 1191 : /*------------------------------------------------------------.
; 1192 : | yynewstate -- Push a new state, which is found in yystate.  |
; 1193 : `------------------------------------------------------------*/
; 1194 :  yynewstate:
; 1195 :   /* In all cases, when you get here, the value and location stacks
; 1196 :      have just been pushed. so pushing a state here evens the stacks.
; 1197 :      */
; 1198 :   yyssp++;

  00081	8b 8d 2c fb ff
	ff		 mov	 ecx, DWORD PTR _yyssp$[ebp]
  00087	83 c1 02	 add	 ecx, 2
  0008a	89 8d 2c fb ff
	ff		 mov	 DWORD PTR _yyssp$[ebp], ecx
$yysetstate$138186:

; 1199 : 
; 1200 :  yysetstate:
; 1201 :   *yyssp = yystate;

  00090	8b 95 2c fb ff
	ff		 mov	 edx, DWORD PTR _yyssp$[ebp]
  00096	66 8b 85 28 fb
	ff ff		 mov	 ax, WORD PTR _yystate$[ebp]
  0009d	66 89 02	 mov	 WORD PTR [edx], ax

; 1202 : 
; 1203 :   if (yyss + yystacksize - 1 <= yyssp)

  000a0	8b 4d fc	 mov	 ecx, DWORD PTR _yystacksize$[ebp]
  000a3	8b 95 c8 fc ff
	ff		 mov	 edx, DWORD PTR _yyss$[ebp]
  000a9	8d 44 4a fe	 lea	 eax, DWORD PTR [edx+ecx*2-2]
  000ad	3b 85 2c fb ff
	ff		 cmp	 eax, DWORD PTR _yyssp$[ebp]
  000b3	0f 87 ee 01 00
	00		 ja	 $yybackup$138234

; 1204 :     {
; 1205 :       /* Get the current used size of the three stacks, in elements.  */
; 1206 :       YYSIZE_T yysize = yyssp - yyss + 1;

  000b9	8b 8d 2c fb ff
	ff		 mov	 ecx, DWORD PTR _yyssp$[ebp]
  000bf	2b 8d c8 fc ff
	ff		 sub	 ecx, DWORD PTR _yyss$[ebp]
  000c5	d1 f9		 sar	 ecx, 1
  000c7	83 c1 01	 add	 ecx, 1
  000ca	89 8d 18 fb ff
	ff		 mov	 DWORD PTR _yysize$138190[ebp], ecx

; 1207 : 
; 1208 : #ifdef yyoverflow
; 1209 :       {
; 1210 :     /* Give user a chance to reallocate the stack. Use copies of
; 1211 :        these so that the &'s don't force the real ones into
; 1212 :        memory.  */
; 1213 :     YYSTYPE *yyvs1 = yyvs;
; 1214 :     short *yyss1 = yyss;
; 1215 : 
; 1216 : 
; 1217 :     /* Each stack pointer address is followed by the size of the
; 1218 :        data in use in that stack, in bytes.  This used to be a
; 1219 :        conditional around just the two extra args, but that might
; 1220 :        be undefined if yyoverflow is a macro.  */
; 1221 :     yyoverflow (_T("parser stack overflow"),
; 1222 :             &yyss1, yysize * sizeof (*yyssp),
; 1223 :             &yyvs1, yysize * sizeof (*yyvsp),
; 1224 : 
; 1225 :             &yystacksize);
; 1226 : 
; 1227 :     yyss = yyss1;
; 1228 :     yyvs = yyvs1;
; 1229 :       }
; 1230 : #else /* no yyoverflow */
; 1231 : # ifndef YYSTACK_RELOCATE
; 1232 :       goto yyoverflowlab;
; 1233 : # else
; 1234 :       /* Extend the stack our own way.  */
; 1235 :       if (YYMAXDEPTH <= yystacksize)

  000d0	81 7d fc 10 27
	00 00		 cmp	 DWORD PTR _yystacksize$[ebp], 10000 ; 00002710H
  000d7	72 0a		 jb	 SHORT $LN99@yyparse
  000d9	e9 30 08 00 00	 jmp	 $yyoverflowlab$138192

; 1236 :     goto yyoverflowlab;

  000de	e9 2b 08 00 00	 jmp	 $yyoverflowlab$138192
$LN99@yyparse:

; 1237 :       yystacksize *= 2;

  000e3	8b 55 fc	 mov	 edx, DWORD PTR _yystacksize$[ebp]
  000e6	d1 e2		 shl	 edx, 1
  000e8	89 55 fc	 mov	 DWORD PTR _yystacksize$[ebp], edx

; 1238 :       if (YYMAXDEPTH < yystacksize)

  000eb	81 7d fc 10 27
	00 00		 cmp	 DWORD PTR _yystacksize$[ebp], 10000 ; 00002710H
  000f2	76 07		 jbe	 SHORT $LN97@yyparse

; 1239 :     yystacksize = YYMAXDEPTH;

  000f4	c7 45 fc 10 27
	00 00		 mov	 DWORD PTR _yystacksize$[ebp], 10000 ; 00002710H
$LN97@yyparse:

; 1240 : 
; 1241 :       {
; 1242 :     short *yyss1 = yyss;

  000fb	8b 85 c8 fc ff
	ff		 mov	 eax, DWORD PTR _yyss$[ebp]
  00101	89 85 14 fb ff
	ff		 mov	 DWORD PTR _yyss1$138195[ebp], eax

; 1243 :     union yyalloc *yyptr =
; 1244 :       (union yyalloc *) YYSTACK_ALLOC (YYSTACK_BYTES (yystacksize));

  00107	8b 45 fc	 mov	 eax, DWORD PTR _yystacksize$[ebp]
  0010a	6b c0 06	 imul	 eax, 6
  0010d	83 c0 03	 add	 eax, 3
  00110	e8 00 00 00 00	 call	 __alloca_probe_16
  00115	89 a5 fc fa ff
	ff		 mov	 DWORD PTR tv79[ebp], esp
  0011b	8b 8d fc fa ff
	ff		 mov	 ecx, DWORD PTR tv79[ebp]
  00121	89 8d 10 fb ff
	ff		 mov	 DWORD PTR _yyptr$138196[ebp], ecx

; 1245 :     if (! yyptr)

  00127	83 bd 10 fb ff
	ff 00		 cmp	 DWORD PTR _yyptr$138196[ebp], 0
  0012e	75 0a		 jne	 SHORT $LN91@yyparse
  00130	e9 d9 07 00 00	 jmp	 $yyoverflowlab$138192

; 1246 :       goto yyoverflowlab;

  00135	e9 d4 07 00 00	 jmp	 $yyoverflowlab$138192
$LN91@yyparse:

; 1247 :     YYSTACK_RELOCATE (yyss);

  0013a	c7 85 08 fb ff
	ff 00 00 00 00	 mov	 DWORD PTR _yyi$138210[ebp], 0
  00144	eb 0f		 jmp	 SHORT $LN88@yyparse
$LN87@yyparse:
  00146	8b 95 08 fb ff
	ff		 mov	 edx, DWORD PTR _yyi$138210[ebp]
  0014c	83 c2 01	 add	 edx, 1
  0014f	89 95 08 fb ff
	ff		 mov	 DWORD PTR _yyi$138210[ebp], edx
$LN88@yyparse:
  00155	8b 85 08 fb ff
	ff		 mov	 eax, DWORD PTR _yyi$138210[ebp]
  0015b	3b 85 18 fb ff
	ff		 cmp	 eax, DWORD PTR _yysize$138190[ebp]
  00161	73 22		 jae	 SHORT $LN90@yyparse
  00163	8b 8d 08 fb ff
	ff		 mov	 ecx, DWORD PTR _yyi$138210[ebp]
  00169	8b 95 10 fb ff
	ff		 mov	 edx, DWORD PTR _yyptr$138196[ebp]
  0016f	8b 85 08 fb ff
	ff		 mov	 eax, DWORD PTR _yyi$138210[ebp]
  00175	8b b5 c8 fc ff
	ff		 mov	 esi, DWORD PTR _yyss$[ebp]
  0017b	66 8b 04 46	 mov	 ax, WORD PTR [esi+eax*2]
  0017f	66 89 04 4a	 mov	 WORD PTR [edx+ecx*2], ax
  00183	eb c1		 jmp	 SHORT $LN87@yyparse
$LN90@yyparse:
  00185	33 c9		 xor	 ecx, ecx
  00187	75 b1		 jne	 SHORT $LN91@yyparse
  00189	8b 95 10 fb ff
	ff		 mov	 edx, DWORD PTR _yyptr$138196[ebp]
  0018f	89 95 c8 fc ff
	ff		 mov	 DWORD PTR _yyss$[ebp], edx
  00195	8b 45 fc	 mov	 eax, DWORD PTR _yystacksize$[ebp]
  00198	8d 4c 00 03	 lea	 ecx, DWORD PTR [eax+eax+3]
  0019c	89 8d 0c fb ff
	ff		 mov	 DWORD PTR _yynewbytes$138206[ebp], ecx
  001a2	8b 95 0c fb ff
	ff		 mov	 edx, DWORD PTR _yynewbytes$138206[ebp]
  001a8	c1 ea 02	 shr	 edx, 2
  001ab	8b 85 10 fb ff
	ff		 mov	 eax, DWORD PTR _yyptr$138196[ebp]
  001b1	8d 0c 90	 lea	 ecx, DWORD PTR [eax+edx*4]
  001b4	89 8d 10 fb ff
	ff		 mov	 DWORD PTR _yyptr$138196[ebp], ecx
  001ba	33 d2		 xor	 edx, edx
  001bc	0f 85 78 ff ff
	ff		 jne	 $LN91@yyparse
$LN82@yyparse:

; 1248 :     YYSTACK_RELOCATE (yyvs);

  001c2	c7 85 00 fb ff
	ff 00 00 00 00	 mov	 DWORD PTR _yyi$138222[ebp], 0
  001cc	eb 0f		 jmp	 SHORT $LN79@yyparse
$LN78@yyparse:
  001ce	8b 85 00 fb ff
	ff		 mov	 eax, DWORD PTR _yyi$138222[ebp]
  001d4	83 c0 01	 add	 eax, 1
  001d7	89 85 00 fb ff
	ff		 mov	 DWORD PTR _yyi$138222[ebp], eax
$LN79@yyparse:
  001dd	8b 8d 00 fb ff
	ff		 mov	 ecx, DWORD PTR _yyi$138222[ebp]
  001e3	3b 8d 18 fb ff
	ff		 cmp	 ecx, DWORD PTR _yysize$138190[ebp]
  001e9	73 20		 jae	 SHORT $LN81@yyparse
  001eb	8b 95 00 fb ff
	ff		 mov	 edx, DWORD PTR _yyi$138222[ebp]
  001f1	8b 85 c4 fc ff
	ff		 mov	 eax, DWORD PTR _yyvs$[ebp]
  001f7	8b 0c 90	 mov	 ecx, DWORD PTR [eax+edx*4]
  001fa	8b 95 00 fb ff
	ff		 mov	 edx, DWORD PTR _yyi$138222[ebp]
  00200	8b 85 10 fb ff
	ff		 mov	 eax, DWORD PTR _yyptr$138196[ebp]
  00206	89 0c 90	 mov	 DWORD PTR [eax+edx*4], ecx
  00209	eb c3		 jmp	 SHORT $LN78@yyparse
$LN81@yyparse:
  0020b	33 c9		 xor	 ecx, ecx
  0020d	75 b3		 jne	 SHORT $LN82@yyparse
  0020f	8b 95 10 fb ff
	ff		 mov	 edx, DWORD PTR _yyptr$138196[ebp]
  00215	89 95 c4 fc ff
	ff		 mov	 DWORD PTR _yyvs$[ebp], edx
  0021b	8b 45 fc	 mov	 eax, DWORD PTR _yystacksize$[ebp]
  0021e	8d 0c 85 03 00
	00 00		 lea	 ecx, DWORD PTR [eax*4+3]
  00225	89 8d 04 fb ff
	ff		 mov	 DWORD PTR _yynewbytes$138218[ebp], ecx
  0022b	8b 95 04 fb ff
	ff		 mov	 edx, DWORD PTR _yynewbytes$138218[ebp]
  00231	c1 ea 02	 shr	 edx, 2
  00234	8b 85 10 fb ff
	ff		 mov	 eax, DWORD PTR _yyptr$138196[ebp]
  0023a	8d 0c 90	 lea	 ecx, DWORD PTR [eax+edx*4]
  0023d	89 8d 10 fb ff
	ff		 mov	 DWORD PTR _yyptr$138196[ebp], ecx
  00243	33 d2		 xor	 edx, edx
  00245	0f 85 77 ff ff
	ff		 jne	 $LN82@yyparse

; 1249 : 
; 1250 : #  undef YYSTACK_RELOCATE
; 1251 :     if (yyss1 != yyssa)

  0024b	8b 85 14 fb ff
	ff		 mov	 eax, DWORD PTR _yyss1$138195[ebp]
  00251	8d 8d 30 fb ff
	ff		 lea	 ecx, DWORD PTR _yyssa$[ebp]
  00257	3b c1		 cmp	 eax, ecx
  00259	74 04		 je	 SHORT $LN76@yyparse
$LN74@yyparse:

; 1252 :       YYSTACK_FREE (yyss1);

  0025b	33 d2		 xor	 edx, edx
  0025d	75 fc		 jne	 SHORT $LN74@yyparse
$LN76@yyparse:

; 1253 :       }
; 1254 : # endif
; 1255 : #endif /* no yyoverflow */
; 1256 : 
; 1257 :       yyssp = yyss + yysize - 1;

  0025f	8b 85 18 fb ff
	ff		 mov	 eax, DWORD PTR _yysize$138190[ebp]
  00265	8b 8d c8 fc ff
	ff		 mov	 ecx, DWORD PTR _yyss$[ebp]
  0026b	8d 54 41 fe	 lea	 edx, DWORD PTR [ecx+eax*2-2]
  0026f	89 95 2c fb ff
	ff		 mov	 DWORD PTR _yyssp$[ebp], edx

; 1258 :       yyvsp = yyvs + yysize - 1;

  00275	8b 85 18 fb ff
	ff		 mov	 eax, DWORD PTR _yysize$138190[ebp]
  0027b	8b 8d c4 fc ff
	ff		 mov	 ecx, DWORD PTR _yyvs$[ebp]
  00281	8d 54 81 fc	 lea	 edx, DWORD PTR [ecx+eax*4-4]
  00285	89 55 f8	 mov	 DWORD PTR _yyvsp$[ebp], edx

; 1259 : 
; 1260 : 
; 1261 :       YYDPRINTF ((stderr, _T("Stack size increased to %lu\n"),
; 1262 :           (unsigned long int) yystacksize));
; 1263 : 
; 1264 :       if (yyss + yystacksize - 1 <= yyssp)

  00288	8b 45 fc	 mov	 eax, DWORD PTR _yystacksize$[ebp]
  0028b	8b 8d c8 fc ff
	ff		 mov	 ecx, DWORD PTR _yyss$[ebp]
  00291	8d 54 41 fe	 lea	 edx, DWORD PTR [ecx+eax*2-2]
  00295	3b 95 2c fb ff
	ff		 cmp	 edx, DWORD PTR _yyssp$[ebp]
  0029b	77 0a		 ja	 SHORT $yybackup$138234
  0029d	e9 5e 06 00 00	 jmp	 $yyabortlab$138232

; 1265 :     YYABORT;

  002a2	e9 59 06 00 00	 jmp	 $yyabortlab$138232
$yybackup$138234:

; 1266 :     }
; 1267 : 
; 1268 :   YYDPRINTF ((stderr, _T("Entering state %d\n"), yystate));
; 1269 : 
; 1270 :   goto yybackup;
; 1271 : 
; 1272 : /*-----------.
; 1273 : | yybackup.  |
; 1274 : `-----------*/
; 1275 : yybackup:
; 1276 : 
; 1277 : /* Do appropriate processing given the current state.  */
; 1278 : /* Read a lookahead token if we need one and don't already have one.  */
; 1279 : /* yyresume: */
; 1280 : 
; 1281 :   /* First try to decide what to do without reference to lookahead token.  */
; 1282 : 
; 1283 :   yyn = yypact[yystate];

  002a7	8b 85 28 fb ff
	ff		 mov	 eax, DWORD PTR _yystate$[ebp]
  002ad	0f bf 0c 45 00
	00 00 00	 movsx	 ecx, WORD PTR _yypact[eax*2]
  002b5	89 8d 20 fb ff
	ff		 mov	 DWORD PTR _yyn$[ebp], ecx

; 1284 :   if (yyn == YYPACT_NINF)

  002bb	81 bd 20 fb ff
	ff 20 ff ff ff	 cmp	 DWORD PTR _yyn$[ebp], -224 ; ffffff20H
  002c5	75 0a		 jne	 SHORT $LN69@yyparse
  002c7	e9 66 01 00 00	 jmp	 $yydefault$138237

; 1285 :     goto yydefault;

  002cc	e9 61 01 00 00	 jmp	 $yydefault$138237
$LN69@yyparse:

; 1286 : 
; 1287 :   /* Not known => get a lookahead token if don't already have one.  */
; 1288 : 
; 1289 :   /* YYCHAR is either YYEMPTY or YYEOF or a valid lookahead symbol.  */
; 1290 :   if (yychar == YYEMPTY)

  002d1	83 3d 00 00 00
	00 fe		 cmp	 DWORD PTR ?yychar@@3HA, -2 ; yychar, fffffffeH
  002d8	75 0a		 jne	 SHORT $LN67@yyparse

; 1291 :     {
; 1292 :       YYDPRINTF ((stderr, _T("Reading a token: ")));
; 1293 :       yychar = YYLEX;

  002da	e8 00 00 00 00	 call	 ?yylex@@YAHXZ		; yylex
  002df	a3 00 00 00 00	 mov	 DWORD PTR ?yychar@@3HA, eax ; yychar
$LN67@yyparse:

; 1294 :     }
; 1295 : 
; 1296 :   if (yychar <= YYEOF)

  002e4	83 3d 00 00 00
	00 00		 cmp	 DWORD PTR ?yychar@@3HA, 0 ; yychar
  002eb	7f 18		 jg	 SHORT $LN66@yyparse

; 1297 :     {
; 1298 :       yychar = yytoken = YYEOF;

  002ed	c7 85 d4 fc ff
	ff 00 00 00 00	 mov	 DWORD PTR _yytoken$[ebp], 0
  002f7	8b 95 d4 fc ff
	ff		 mov	 edx, DWORD PTR _yytoken$[ebp]
  002fd	89 15 00 00 00
	00		 mov	 DWORD PTR ?yychar@@3HA, edx ; yychar

; 1299 :       YYDPRINTF ((stderr, _T("Now at end of input.\n")));
; 1300 :     }
; 1301 :   else

  00303	eb 36		 jmp	 SHORT $LN65@yyparse
$LN66@yyparse:

; 1302 :     {
; 1303 :       yytoken = YYTRANSLATE (yychar);

  00305	81 3d 00 00 00
	00 38 01 00 00	 cmp	 DWORD PTR ?yychar@@3HA, 312 ; yychar, 00000138H
  0030f	77 14		 ja	 SHORT $LN104@yyparse
  00311	a1 00 00 00 00	 mov	 eax, DWORD PTR ?yychar@@3HA ; yychar
  00316	0f b6 88 00 00
	00 00		 movzx	 ecx, BYTE PTR _yytranslate[eax]
  0031d	89 8d f8 fa ff
	ff		 mov	 DWORD PTR tv162[ebp], ecx
  00323	eb 0a		 jmp	 SHORT $LN105@yyparse
$LN104@yyparse:
  00325	c7 85 f8 fa ff
	ff 02 00 00 00	 mov	 DWORD PTR tv162[ebp], 2
$LN105@yyparse:
  0032f	8b 95 f8 fa ff
	ff		 mov	 edx, DWORD PTR tv162[ebp]
  00335	89 95 d4 fc ff
	ff		 mov	 DWORD PTR _yytoken$[ebp], edx
$LN65@yyparse:

; 1304 :       YYDSYMPRINTF (_T("Next token is"), yytoken, &yylval, &yylloc);
; 1305 :     }
; 1306 : 
; 1307 :   /* If the proper action on seeing token YYTOKEN is to reduce or to
; 1308 :      detect an error, take that action.  */
; 1309 :   yyn += yytoken;

  0033b	8b 85 20 fb ff
	ff		 mov	 eax, DWORD PTR _yyn$[ebp]
  00341	03 85 d4 fc ff
	ff		 add	 eax, DWORD PTR _yytoken$[ebp]
  00347	89 85 20 fb ff
	ff		 mov	 DWORD PTR _yyn$[ebp], eax

; 1310 :   if (yyn < 0 || YYLAST < yyn || yycheck[yyn] != yytoken)

  0034d	78 22		 js	 SHORT $LN63@yyparse
  0034f	81 bd 20 fb ff
	ff 2e 01 00 00	 cmp	 DWORD PTR _yyn$[ebp], 302 ; 0000012eH
  00359	7f 16		 jg	 SHORT $LN63@yyparse
  0035b	8b 8d 20 fb ff
	ff		 mov	 ecx, DWORD PTR _yyn$[ebp]
  00361	0f bf 14 4d 00
	00 00 00	 movsx	 edx, WORD PTR _yycheck[ecx*2]
  00369	3b 95 d4 fc ff
	ff		 cmp	 edx, DWORD PTR _yytoken$[ebp]
  0036f	74 0a		 je	 SHORT $LN64@yyparse
$LN63@yyparse:

; 1311 :     goto yydefault;

  00371	e9 bc 00 00 00	 jmp	 $yydefault$138237
  00376	e9 b7 00 00 00	 jmp	 $yydefault$138237
$LN64@yyparse:

; 1312 :   yyn = yytable[yyn];

  0037b	8b 85 20 fb ff
	ff		 mov	 eax, DWORD PTR _yyn$[ebp]
  00381	0f bf 0c 45 00
	00 00 00	 movsx	 ecx, WORD PTR _yytable[eax*2]
  00389	89 8d 20 fb ff
	ff		 mov	 DWORD PTR _yyn$[ebp], ecx

; 1313 :   if (yyn <= 0)

  0038f	83 bd 20 fb ff
	ff 00		 cmp	 DWORD PTR _yyn$[ebp], 0
  00396	7f 37		 jg	 SHORT $LN61@yyparse

; 1314 :     {
; 1315 :       if (yyn == 0 || yyn == YYTABLE_NINF)

  00398	83 bd 20 fb ff
	ff 00		 cmp	 DWORD PTR _yyn$[ebp], 0
  0039f	74 0c		 je	 SHORT $LN59@yyparse
  003a1	81 bd 20 fb ff
	ff 79 ff ff ff	 cmp	 DWORD PTR _yyn$[ebp], -135 ; ffffff79H
  003ab	75 0a		 jne	 SHORT $LN60@yyparse
$LN59@yyparse:

; 1316 :     goto yyerrlab;

  003ad	e9 78 03 00 00	 jmp	 $yyerrlab$138249
  003b2	e9 73 03 00 00	 jmp	 $yyerrlab$138249
$LN60@yyparse:

; 1317 :       yyn = -yyn;

  003b7	8b 95 20 fb ff
	ff		 mov	 edx, DWORD PTR _yyn$[ebp]
  003bd	f7 da		 neg	 edx
  003bf	89 95 20 fb ff
	ff		 mov	 DWORD PTR _yyn$[ebp], edx
  003c5	e9 8e 00 00 00	 jmp	 $yyreduce$138251

; 1318 :       goto yyreduce;

  003ca	e9 89 00 00 00	 jmp	 $yyreduce$138251
$LN61@yyparse:

; 1319 :     }
; 1320 : 
; 1321 :   if (yyn == YYFINAL)

  003cf	83 bd 20 fb ff
	ff 0c		 cmp	 DWORD PTR _yyn$[ebp], 12 ; 0000000cH
  003d6	75 0a		 jne	 SHORT $LN56@yyparse
  003d8	e9 15 05 00 00	 jmp	 $yyacceptlab$138254

; 1322 :     YYACCEPT;

  003dd	e9 10 05 00 00	 jmp	 $yyacceptlab$138254
$LN56@yyparse:

; 1323 : 
; 1324 :   /* Shift the lookahead token.  */
; 1325 :   YYDPRINTF ((stderr, _T("Shifting token %s, "), yytname[yytoken]));
; 1326 : 
; 1327 :   /* Discard the token being shifted unless it is eof.  */
; 1328 :   if (yychar != YYEOF)

  003e2	83 3d 00 00 00
	00 00		 cmp	 DWORD PTR ?yychar@@3HA, 0 ; yychar
  003e9	74 0a		 je	 SHORT $LN54@yyparse

; 1329 :     yychar = YYEMPTY;

  003eb	c7 05 00 00 00
	00 fe ff ff ff	 mov	 DWORD PTR ?yychar@@3HA, -2 ; yychar, fffffffeH
$LN54@yyparse:

; 1330 : 
; 1331 :   *++yyvsp = yylval;

  003f5	8b 45 f8	 mov	 eax, DWORD PTR _yyvsp$[ebp]
  003f8	83 c0 04	 add	 eax, 4
  003fb	89 45 f8	 mov	 DWORD PTR _yyvsp$[ebp], eax
  003fe	8b 4d f8	 mov	 ecx, DWORD PTR _yyvsp$[ebp]
  00401	8b 15 00 00 00
	00		 mov	 edx, DWORD PTR ?yylval@@3TYYSTYPE@@A ; yylval
  00407	89 11		 mov	 DWORD PTR [ecx], edx

; 1332 : 
; 1333 : 
; 1334 :   /* Count tokens shifted since error; after three, turn off error
; 1335 :      status.  */
; 1336 :   if (yyerrstatus)

  00409	83 bd 1c fb ff
	ff 00		 cmp	 DWORD PTR _yyerrstatus$[ebp], 0
  00410	74 0f		 je	 SHORT $LN53@yyparse

; 1337 :     yyerrstatus--;

  00412	8b 85 1c fb ff
	ff		 mov	 eax, DWORD PTR _yyerrstatus$[ebp]
  00418	83 e8 01	 sub	 eax, 1
  0041b	89 85 1c fb ff
	ff		 mov	 DWORD PTR _yyerrstatus$[ebp], eax
$LN53@yyparse:

; 1338 : 
; 1339 :   yystate = yyn;

  00421	8b 8d 20 fb ff
	ff		 mov	 ecx, DWORD PTR _yyn$[ebp]
  00427	89 8d 28 fb ff
	ff		 mov	 DWORD PTR _yystate$[ebp], ecx
  0042d	e9 4f fc ff ff	 jmp	 $yynewstate$138188
$yydefault$138237:

; 1340 :   goto yynewstate;
; 1341 : 
; 1342 : 
; 1343 : /*-----------------------------------------------------------.
; 1344 : | yydefault -- do the default action for the current state.  |
; 1345 : `-----------------------------------------------------------*/
; 1346 : yydefault:
; 1347 :   yyn = yydefact[yystate];

  00432	8b 95 28 fb ff
	ff		 mov	 edx, DWORD PTR _yystate$[ebp]
  00438	0f b6 82 00 00
	00 00		 movzx	 eax, BYTE PTR _yydefact[edx]
  0043f	89 85 20 fb ff
	ff		 mov	 DWORD PTR _yyn$[ebp], eax

; 1348 :   if (yyn == 0)

  00445	83 bd 20 fb ff
	ff 00		 cmp	 DWORD PTR _yyn$[ebp], 0
  0044c	75 0a		 jne	 SHORT $yyreduce$138251
  0044e	e9 d7 02 00 00	 jmp	 $yyerrlab$138249

; 1349 :     goto yyerrlab;

  00453	e9 d2 02 00 00	 jmp	 $yyerrlab$138249
$yyreduce$138251:

; 1350 :   goto yyreduce;
; 1351 : 
; 1352 : 
; 1353 : /*-----------------------------.
; 1354 : | yyreduce -- Do a reduction.  |
; 1355 : `-----------------------------*/
; 1356 : yyreduce:
; 1357 :   /* yyn is the number of a rule to reduce with.  */
; 1358 :   yylen = yyr2[yyn];

  00458	8b 8d 20 fb ff
	ff		 mov	 ecx, DWORD PTR _yyn$[ebp]
  0045e	0f b6 91 00 00
	00 00		 movzx	 edx, BYTE PTR _yyr2[ecx]
  00465	89 95 d0 fc ff
	ff		 mov	 DWORD PTR _yylen$[ebp], edx

; 1359 : 
; 1360 :   /* If YYLEN is nonzero, implement the default value of the action:
; 1361 :      `$$ = $1'.
; 1362 : 
; 1363 :      Otherwise, the following line sets YYVAL to garbage.
; 1364 :      This behavior is undocumented and Bison
; 1365 :      users should not rely upon it.  Assigning to YYVAL
; 1366 :      unconditionally makes the parser a bit smaller, and it avoids a
; 1367 :      GCC warning that YYVAL may be used uninitialized.  */
; 1368 :   yyval = yyvsp[1-yylen];

  0046b	b8 01 00 00 00	 mov	 eax, 1
  00470	2b 85 d0 fc ff
	ff		 sub	 eax, DWORD PTR _yylen$[ebp]
  00476	8b 4d f8	 mov	 ecx, DWORD PTR _yyvsp$[ebp]
  00479	8b 14 81	 mov	 edx, DWORD PTR [ecx+eax*4]
  0047c	89 95 cc fc ff
	ff		 mov	 DWORD PTR _yyval$[ebp], edx

; 1369 : 
; 1370 : 
; 1371 :   YY_REDUCE_PRINT (yyn);
; 1372 :   switch (yyn)

  00482	8b 85 20 fb ff
	ff		 mov	 eax, DWORD PTR _yyn$[ebp]
  00488	89 85 f4 fa ff
	ff		 mov	 DWORD PTR tv191[ebp], eax
  0048e	8b 8d f4 fa ff
	ff		 mov	 ecx, DWORD PTR tv191[ebp]
  00494	83 e9 18	 sub	 ecx, 24			; 00000018H
  00497	89 8d f4 fa ff
	ff		 mov	 DWORD PTR tv191[ebp], ecx
  0049d	83 bd f4 fa ff
	ff 7c		 cmp	 DWORD PTR tv191[ebp], 124 ; 0000007cH
  004a4	0f 87 bb 01 00
	00		 ja	 $LN48@yyparse
  004aa	8b 95 f4 fa ff
	ff		 mov	 edx, DWORD PTR tv191[ebp]
  004b0	0f b6 82 00 00
	00 00		 movzx	 eax, BYTE PTR $LN106@yyparse[edx]
  004b7	ff 24 85 00 00
	00 00		 jmp	 DWORD PTR $LN107@yyparse[eax*4]
$LN47@yyparse:

; 1373 :     {
; 1374 :         case 24:
; 1375 : //#line 94 _T("xml_prolog.yy")
; 1376 :     { XmltvTags_PiContent(NULL); }

  004be	6a 00		 push	 0
  004c0	e8 00 00 00 00	 call	 ?XmltvTags_PiContent@@YAXPB_W@Z ; XmltvTags_PiContent
  004c5	83 c4 04	 add	 esp, 4

; 1377 :     break;

  004c8	e9 98 01 00 00	 jmp	 $LN48@yyparse
$LN46@yyparse:

; 1378 : 
; 1379 :   case 31:
; 1380 : //#line 102 _T("xml_prolog.yy")
; 1381 :     {XmltvTags_DocIntDtdClose();}

  004cd	e8 00 00 00 00	 call	 ?XmltvTags_DocIntDtdClose@@YAXXZ ; XmltvTags_DocIntDtdClose

; 1382 :     break;

  004d2	e9 8e 01 00 00	 jmp	 $LN48@yyparse
$LN45@yyparse:

; 1383 : 
; 1384 :   case 32:
; 1385 : //#line 103 _T("xml_prolog.yy")
; 1386 :     {XmltvTags_DocIntDtdClose();}

  004d7	e8 00 00 00 00	 call	 ?XmltvTags_DocIntDtdClose@@YAXXZ ; XmltvTags_DocIntDtdClose

; 1387 :     break;

  004dc	e9 84 01 00 00	 jmp	 $LN48@yyparse
$LN44@yyparse:

; 1388 : 
; 1389 :   case 45:
; 1390 : //#line 122 _T("xml_prolog.yy")
; 1391 :     {yyerrok;}

  004e1	c7 85 1c fb ff
	ff 00 00 00 00	 mov	 DWORD PTR _yyerrstatus$[ebp], 0

; 1392 :     break;

  004eb	e9 75 01 00 00	 jmp	 $LN48@yyparse
$LN43@yyparse:

; 1393 : 
; 1394 :   case 46:
; 1395 : //#line 123 _T("xml_prolog.yy")
; 1396 :     {yyerrok;}

  004f0	c7 85 1c fb ff
	ff 00 00 00 00	 mov	 DWORD PTR _yyerrstatus$[ebp], 0

; 1397 :     break;

  004fa	e9 66 01 00 00	 jmp	 $LN48@yyparse
$LN42@yyparse:

; 1398 : 
; 1399 :   case 121:
; 1400 : //#line 189 _T("xml_prolog.yy")
; 1401 :     {XmltvTags_Notation(1, yyvsp[-1].str);}

  004ff	8b 4d f8	 mov	 ecx, DWORD PTR _yyvsp$[ebp]
  00502	8b 51 fc	 mov	 edx, DWORD PTR [ecx-4]
  00505	52		 push	 edx
  00506	6a 01		 push	 1
  00508	e8 00 00 00 00	 call	 ?XmltvTags_Notation@@YAXHPB_W@Z ; XmltvTags_Notation
  0050d	83 c4 08	 add	 esp, 8

; 1402 :     break;

  00510	e9 50 01 00 00	 jmp	 $LN48@yyparse
$LN41@yyparse:

; 1403 : 
; 1404 :   case 122:
; 1405 : //#line 190 _T("xml_prolog.yy")
; 1406 :     {XmltvTags_Notation(2, yyvsp[-1].str);}

  00515	8b 45 f8	 mov	 eax, DWORD PTR _yyvsp$[ebp]
  00518	8b 48 fc	 mov	 ecx, DWORD PTR [eax-4]
  0051b	51		 push	 ecx
  0051c	6a 02		 push	 2
  0051e	e8 00 00 00 00	 call	 ?XmltvTags_Notation@@YAXHPB_W@Z ; XmltvTags_Notation
  00523	83 c4 08	 add	 esp, 8

; 1407 :     break;

  00526	e9 3a 01 00 00	 jmp	 $LN48@yyparse
$LN40@yyparse:

; 1408 : 
; 1409 :   case 123:
; 1410 : //#line 190 _T("xml_prolog.yy")
; 1411 :     {XmltvTags_Notation(4, yyvsp[0].str);}

  0052b	8b 55 f8	 mov	 edx, DWORD PTR _yyvsp$[ebp]
  0052e	8b 02		 mov	 eax, DWORD PTR [edx]
  00530	50		 push	 eax
  00531	6a 04		 push	 4
  00533	e8 00 00 00 00	 call	 ?XmltvTags_Notation@@YAXHPB_W@Z ; XmltvTags_Notation
  00538	83 c4 08	 add	 esp, 8

; 1412 :     break;

  0053b	e9 25 01 00 00	 jmp	 $LN48@yyparse
$LN39@yyparse:

; 1413 : 
; 1414 :   case 125:
; 1415 : //#line 191 _T("xml_prolog.yy")
; 1416 :     {XmltvTags_Notation(3, yyvsp[-1].str);}

  00540	8b 4d f8	 mov	 ecx, DWORD PTR _yyvsp$[ebp]
  00543	8b 51 fc	 mov	 edx, DWORD PTR [ecx-4]
  00546	52		 push	 edx
  00547	6a 03		 push	 3
  00549	e8 00 00 00 00	 call	 ?XmltvTags_Notation@@YAXHPB_W@Z ; XmltvTags_Notation
  0054e	83 c4 08	 add	 esp, 8

; 1417 :     break;

  00551	e9 0f 01 00 00	 jmp	 $LN48@yyparse
$LN38@yyparse:

; 1418 : 
; 1419 :   case 135:
; 1420 : //#line 203 _T("xml_prolog.yy")
; 1421 :     { XmltvTags_Encoding(yyvsp[0].str); }

  00556	8b 45 f8	 mov	 eax, DWORD PTR _yyvsp$[ebp]
  00559	8b 08		 mov	 ecx, DWORD PTR [eax]
  0055b	51		 push	 ecx
  0055c	e8 00 00 00 00	 call	 ?XmltvTags_Encoding@@YAXPB_W@Z ; XmltvTags_Encoding
  00561	83 c4 04	 add	 esp, 4

; 1422 :     break;

  00564	e9 fc 00 00 00	 jmp	 $LN48@yyparse
$LN37@yyparse:

; 1423 : 
; 1424 :   case 136:
; 1425 : //#line 204 _T("xml_prolog.yy")
; 1426 :     { XmltvTags_XmlVersion(yyvsp[0].str); }

  00569	8b 55 f8	 mov	 edx, DWORD PTR _yyvsp$[ebp]
  0056c	8b 02		 mov	 eax, DWORD PTR [edx]
  0056e	50		 push	 eax
  0056f	e8 00 00 00 00	 call	 ?XmltvTags_XmlVersion@@YAXPB_W@Z ; XmltvTags_XmlVersion
  00574	83 c4 04	 add	 esp, 4

; 1427 :     break;

  00577	e9 e9 00 00 00	 jmp	 $LN48@yyparse
$LN36@yyparse:

; 1428 : 
; 1429 :   case 137:
; 1430 : //#line 205 _T("xml_prolog.yy")
; 1431 :     { XmltvTags_DocType(yyvsp[0].str); }

  0057c	8b 4d f8	 mov	 ecx, DWORD PTR _yyvsp$[ebp]
  0057f	8b 11		 mov	 edx, DWORD PTR [ecx]
  00581	52		 push	 edx
  00582	e8 00 00 00 00	 call	 ?XmltvTags_DocType@@YAXPB_W@Z ; XmltvTags_DocType
  00587	83 c4 04	 add	 esp, 4

; 1432 :     break;

  0058a	e9 d6 00 00 00	 jmp	 $LN48@yyparse
$LN35@yyparse:

; 1433 : 
; 1434 :   case 138:
; 1435 : //#line 206 _T("xml_prolog.yy")
; 1436 :     { XmlScan_EntityDefName(yyvsp[0].str, 0); XmltvTags_CheckName(yyvsp[0].str); }

  0058f	6a 00		 push	 0
  00591	8b 45 f8	 mov	 eax, DWORD PTR _yyvsp$[ebp]
  00594	8b 08		 mov	 ecx, DWORD PTR [eax]
  00596	51		 push	 ecx
  00597	e8 00 00 00 00	 call	 ?XmlScan_EntityDefName@@YAXPB_WH@Z ; XmlScan_EntityDefName
  0059c	83 c4 08	 add	 esp, 8
  0059f	8b 55 f8	 mov	 edx, DWORD PTR _yyvsp$[ebp]
  005a2	8b 02		 mov	 eax, DWORD PTR [edx]
  005a4	50		 push	 eax
  005a5	e8 00 00 00 00	 call	 ?XmltvTags_CheckName@@YAXPB_W@Z ; XmltvTags_CheckName
  005aa	83 c4 04	 add	 esp, 4

; 1437 :     break;

  005ad	e9 b3 00 00 00	 jmp	 $LN48@yyparse
$LN34@yyparse:

; 1438 : 
; 1439 :   case 139:
; 1440 : //#line 207 _T("xml_prolog.yy")
; 1441 :     { XmlScan_EntityDefName(yyvsp[0].str, 1); XmltvTags_CheckName(yyvsp[0].str); }

  005b2	6a 01		 push	 1
  005b4	8b 4d f8	 mov	 ecx, DWORD PTR _yyvsp$[ebp]
  005b7	8b 11		 mov	 edx, DWORD PTR [ecx]
  005b9	52		 push	 edx
  005ba	e8 00 00 00 00	 call	 ?XmlScan_EntityDefName@@YAXPB_WH@Z ; XmlScan_EntityDefName
  005bf	83 c4 08	 add	 esp, 8
  005c2	8b 45 f8	 mov	 eax, DWORD PTR _yyvsp$[ebp]
  005c5	8b 08		 mov	 ecx, DWORD PTR [eax]
  005c7	51		 push	 ecx
  005c8	e8 00 00 00 00	 call	 ?XmltvTags_CheckName@@YAXPB_W@Z ; XmltvTags_CheckName
  005cd	83 c4 04	 add	 esp, 4

; 1442 :     break;

  005d0	e9 90 00 00 00	 jmp	 $LN48@yyparse
$LN33@yyparse:

; 1443 : 
; 1444 :   case 140:
; 1445 : //#line 208 _T("xml_prolog.yy")
; 1446 :     { XmlScan_EntityDefValue(yyvsp[0].str); XmltvTags_CheckCharset(yyvsp[0].str); }

  005d5	8b 55 f8	 mov	 edx, DWORD PTR _yyvsp$[ebp]
  005d8	8b 02		 mov	 eax, DWORD PTR [edx]
  005da	50		 push	 eax
  005db	e8 00 00 00 00	 call	 ?XmlScan_EntityDefValue@@YAXPB_W@Z ; XmlScan_EntityDefValue
  005e0	83 c4 04	 add	 esp, 4
  005e3	8b 4d f8	 mov	 ecx, DWORD PTR _yyvsp$[ebp]
  005e6	8b 11		 mov	 edx, DWORD PTR [ecx]
  005e8	52		 push	 edx
  005e9	e8 00 00 00 00	 call	 ?XmltvTags_CheckCharset@@YAXPB_W@Z ; XmltvTags_CheckCharset
  005ee	83 c4 04	 add	 esp, 4

; 1447 :     break;

  005f1	eb 72		 jmp	 SHORT $LN48@yyparse
$LN32@yyparse:

; 1448 : 
; 1449 :   case 141:
; 1450 : //#line 210 _T("xml_prolog.yy")
; 1451 :     { XmltvTags_Notation(0, yyvsp[0].str); }

  005f3	8b 45 f8	 mov	 eax, DWORD PTR _yyvsp$[ebp]
  005f6	8b 08		 mov	 ecx, DWORD PTR [eax]
  005f8	51		 push	 ecx
  005f9	6a 00		 push	 0
  005fb	e8 00 00 00 00	 call	 ?XmltvTags_Notation@@YAXHPB_W@Z ; XmltvTags_Notation
  00600	83 c4 08	 add	 esp, 8

; 1452 :     break;

  00603	eb 60		 jmp	 SHORT $LN48@yyparse

; 1453 : 
; 1454 :   case 142:
; 1455 : //#line 211 _T("xml_prolog.yy")
; 1456 :     { }
; 1457 :     break;

  00605	eb 5e		 jmp	 SHORT $LN48@yyparse
$LN30@yyparse:

; 1458 : 
; 1459 :   case 143:
; 1460 : //#line 212 _T("xml_prolog.yy")
; 1461 :     { XmltvTags_PiTarget(yyvsp[0].str); }

  00607	8b 55 f8	 mov	 edx, DWORD PTR _yyvsp$[ebp]
  0060a	8b 02		 mov	 eax, DWORD PTR [edx]
  0060c	50		 push	 eax
  0060d	e8 00 00 00 00	 call	 ?XmltvTags_PiTarget@@YAXPB_W@Z ; XmltvTags_PiTarget
  00612	83 c4 04	 add	 esp, 4

; 1462 :     break;

  00615	eb 4e		 jmp	 SHORT $LN48@yyparse
$LN29@yyparse:

; 1463 : 
; 1464 :   case 144:
; 1465 : //#line 213 _T("xml_prolog.yy")
; 1466 :     { XmltvTags_PiContent(yyvsp[0].str); }

  00617	8b 4d f8	 mov	 ecx, DWORD PTR _yyvsp$[ebp]
  0061a	8b 11		 mov	 edx, DWORD PTR [ecx]
  0061c	52		 push	 edx
  0061d	e8 00 00 00 00	 call	 ?XmltvTags_PiContent@@YAXPB_W@Z ; XmltvTags_PiContent
  00622	83 c4 04	 add	 esp, 4

; 1467 :     break;

  00625	eb 3e		 jmp	 SHORT $LN48@yyparse
$LN28@yyparse:

; 1468 : 
; 1469 :   case 145:
; 1470 : //#line 215 _T("xml_prolog.yy")
; 1471 :     { XmltvTags_CheckName(yyvsp[0].str); }

  00627	8b 45 f8	 mov	 eax, DWORD PTR _yyvsp$[ebp]
  0062a	8b 08		 mov	 ecx, DWORD PTR [eax]
  0062c	51		 push	 ecx
  0062d	e8 00 00 00 00	 call	 ?XmltvTags_CheckName@@YAXPB_W@Z ; XmltvTags_CheckName
  00632	83 c4 04	 add	 esp, 4

; 1472 :     break;

  00635	eb 2e		 jmp	 SHORT $LN48@yyparse
$LN27@yyparse:

; 1473 : 
; 1474 :   case 146:
; 1475 : //#line 216 _T("xml_prolog.yy")
; 1476 :     { XmltvTags_CheckNmtoken(yyvsp[0].str); }

  00637	8b 55 f8	 mov	 edx, DWORD PTR _yyvsp$[ebp]
  0063a	8b 02		 mov	 eax, DWORD PTR [edx]
  0063c	50		 push	 eax
  0063d	e8 00 00 00 00	 call	 ?XmltvTags_CheckNmtoken@@YAXPB_W@Z ; XmltvTags_CheckNmtoken
  00642	83 c4 04	 add	 esp, 4

; 1477 :     break;

  00645	eb 1e		 jmp	 SHORT $LN48@yyparse
$LN26@yyparse:

; 1478 : 
; 1479 :   case 147:
; 1480 : //#line 217 _T("xml_prolog.yy")
; 1481 :     { XmltvTags_CheckSystemLiteral(yyvsp[0].str); }

  00647	8b 4d f8	 mov	 ecx, DWORD PTR _yyvsp$[ebp]
  0064a	8b 11		 mov	 edx, DWORD PTR [ecx]
  0064c	52		 push	 edx
  0064d	e8 00 00 00 00	 call	 ?XmltvTags_CheckSystemLiteral@@YAXPB_W@Z ; XmltvTags_CheckSystemLiteral
  00652	83 c4 04	 add	 esp, 4

; 1482 :     break;

  00655	eb 0e		 jmp	 SHORT $LN48@yyparse
$LN25@yyparse:

; 1483 : 
; 1484 :   case 148:
; 1485 : //#line 218 _T("xml_prolog.yy")
; 1486 :     { XmltvTags_CheckCharset(yyvsp[0].str); }

  00657	8b 45 f8	 mov	 eax, DWORD PTR _yyvsp$[ebp]
  0065a	8b 08		 mov	 ecx, DWORD PTR [eax]
  0065c	51		 push	 ecx
  0065d	e8 00 00 00 00	 call	 ?XmltvTags_CheckCharset@@YAXPB_W@Z ; XmltvTags_CheckCharset
  00662	83 c4 04	 add	 esp, 4
$LN48@yyparse:

; 1487 :     break;
; 1488 : 
; 1489 : 
; 1490 :     }
; 1491 : 
; 1492 : /* Line 991 of yacc.c.  */
; 1493 : //#line 1497 _T("xml_prolog.tab.c")
; 1494 : 
; 1495 :   yyvsp -= yylen;

  00665	8b 95 d0 fc ff
	ff		 mov	 edx, DWORD PTR _yylen$[ebp]
  0066b	c1 e2 02	 shl	 edx, 2
  0066e	8b 45 f8	 mov	 eax, DWORD PTR _yyvsp$[ebp]
  00671	2b c2		 sub	 eax, edx
  00673	89 45 f8	 mov	 DWORD PTR _yyvsp$[ebp], eax

; 1496 :   yyssp -= yylen;

  00676	8b 8d d0 fc ff
	ff		 mov	 ecx, DWORD PTR _yylen$[ebp]
  0067c	d1 e1		 shl	 ecx, 1
  0067e	8b 95 2c fb ff
	ff		 mov	 edx, DWORD PTR _yyssp$[ebp]
  00684	2b d1		 sub	 edx, ecx
  00686	89 95 2c fb ff
	ff		 mov	 DWORD PTR _yyssp$[ebp], edx

; 1497 : 
; 1498 : 
; 1499 :   YY_STACK_PRINT (yyss, yyssp);
; 1500 : 
; 1501 :   *++yyvsp = yyval;

  0068c	8b 45 f8	 mov	 eax, DWORD PTR _yyvsp$[ebp]
  0068f	83 c0 04	 add	 eax, 4
  00692	89 45 f8	 mov	 DWORD PTR _yyvsp$[ebp], eax
  00695	8b 4d f8	 mov	 ecx, DWORD PTR _yyvsp$[ebp]
  00698	8b 95 cc fc ff
	ff		 mov	 edx, DWORD PTR _yyval$[ebp]
  0069e	89 11		 mov	 DWORD PTR [ecx], edx

; 1502 : 
; 1503 : 
; 1504 :   /* Now `shift' the result of the reduction.  Determine what state
; 1505 :      that goes to, based on the state we popped back to and the rule
; 1506 :      number reduced by.  */
; 1507 : 
; 1508 :   yyn = yyr1[yyn];

  006a0	8b 85 20 fb ff
	ff		 mov	 eax, DWORD PTR _yyn$[ebp]
  006a6	0f b6 88 00 00
	00 00		 movzx	 ecx, BYTE PTR _yyr1[eax]
  006ad	89 8d 20 fb ff
	ff		 mov	 DWORD PTR _yyn$[ebp], ecx

; 1509 : 
; 1510 :   yystate = yypgoto[yyn - YYNTOKENS] + *yyssp;

  006b3	8b 95 20 fb ff
	ff		 mov	 edx, DWORD PTR _yyn$[ebp]
  006b9	0f bf 04 55 8c
	ff ff ff	 movsx	 eax, WORD PTR _yypgoto[edx*2-116]
  006c1	8b 8d 2c fb ff
	ff		 mov	 ecx, DWORD PTR _yyssp$[ebp]
  006c7	0f bf 11	 movsx	 edx, WORD PTR [ecx]
  006ca	03 c2		 add	 eax, edx
  006cc	89 85 28 fb ff
	ff		 mov	 DWORD PTR _yystate$[ebp], eax

; 1511 :   if (0 <= yystate && yystate <= YYLAST && yycheck[yystate] == *yyssp)

  006d2	78 3d		 js	 SHORT $LN24@yyparse
  006d4	81 bd 28 fb ff
	ff 2e 01 00 00	 cmp	 DWORD PTR _yystate$[ebp], 302 ; 0000012eH
  006de	7f 31		 jg	 SHORT $LN24@yyparse
  006e0	8b 85 28 fb ff
	ff		 mov	 eax, DWORD PTR _yystate$[ebp]
  006e6	0f bf 0c 45 00
	00 00 00	 movsx	 ecx, WORD PTR _yycheck[eax*2]
  006ee	8b 95 2c fb ff
	ff		 mov	 edx, DWORD PTR _yyssp$[ebp]
  006f4	0f bf 02	 movsx	 eax, WORD PTR [edx]
  006f7	3b c8		 cmp	 ecx, eax
  006f9	75 16		 jne	 SHORT $LN24@yyparse

; 1512 :     yystate = yytable[yystate];

  006fb	8b 8d 28 fb ff
	ff		 mov	 ecx, DWORD PTR _yystate$[ebp]
  00701	0f bf 14 4d 00
	00 00 00	 movsx	 edx, WORD PTR _yytable[ecx*2]
  00709	89 95 28 fb ff
	ff		 mov	 DWORD PTR _yystate$[ebp], edx

; 1513 :   else

  0070f	eb 14		 jmp	 SHORT $LN23@yyparse
$LN24@yyparse:

; 1514 :     yystate = yydefgoto[yyn - YYNTOKENS];

  00711	8b 85 20 fb ff
	ff		 mov	 eax, DWORD PTR _yyn$[ebp]
  00717	0f bf 0c 45 8c
	ff ff ff	 movsx	 ecx, WORD PTR _yydefgoto[eax*2-116]
  0071f	89 8d 28 fb ff
	ff		 mov	 DWORD PTR _yystate$[ebp], ecx
$LN23@yyparse:
  00725	e9 57 f9 ff ff	 jmp	 $yynewstate$138188
$yyerrlab$138249:

; 1515 : 
; 1516 :   goto yynewstate;
; 1517 : 
; 1518 : 
; 1519 : /*------------------------------------.
; 1520 : | yyerrlab -- here on detecting error |
; 1521 : `------------------------------------*/
; 1522 : yyerrlab:
; 1523 :   /* If not already recovering from an error, report this error.  */
; 1524 :   if (!yyerrstatus)

  0072a	83 bd 1c fb ff
	ff 00		 cmp	 DWORD PTR _yyerrstatus$[ebp], 0
  00731	75 1c		 jne	 SHORT $LN22@yyparse

; 1525 :     {
; 1526 :       ++yynerrs;

  00733	8b 15 00 00 00
	00		 mov	 edx, DWORD PTR ?yynerrs@@3HA ; yynerrs
  00739	83 c2 01	 add	 edx, 1
  0073c	89 15 00 00 00
	00		 mov	 DWORD PTR ?yynerrs@@3HA, edx ; yynerrs

; 1527 : #if YYERROR_VERBOSE
; 1528 :       yyn = yypact[yystate];
; 1529 : 
; 1530 :       if (YYPACT_NINF < yyn && yyn < YYLAST)
; 1531 :     {
; 1532 :       YYSIZE_T yysize = 0;
; 1533 :       int yytype = YYTRANSLATE (yychar);
; 1534 :       TCHAR* yymsg;
; 1535 :       int yyx, yycount;
; 1536 : 
; 1537 :       yycount = 0;
; 1538 :       /* Start YYX at -YYN if negative to avoid negative indexes in
; 1539 :          YYCHECK.  */
; 1540 :       for (yyx = yyn < 0 ? -yyn : 0;
; 1541 :            yyx < (int) (sizeof (yytname) / sizeof (TCHAR* )); yyx++)
; 1542 :         if (yycheck[yyx + yyn] == yyx && yyx != YYTERROR)
; 1543 :           yysize += yystrlen (yytname[yyx]) + 15, yycount++;
; 1544 :       yysize += yystrlen (_T("syntax error, unexpected ")) + 1;
; 1545 :       yysize += yystrlen (yytname[yytype]);
; 1546 :       yymsg = (TCHAR* ) YYSTACK_ALLOC (yysize);
; 1547 :       if (yymsg != 0)
; 1548 :         {
; 1549 :           TCHAR* yyp = yystpcpy (yymsg, _T("syntax error, unexpected "));
; 1550 :           yyp = yystpcpy (yyp, yytname[yytype]);
; 1551 : 
; 1552 :           if (yycount < 5)
; 1553 :         {
; 1554 :           yycount = 0;
; 1555 :           for (yyx = yyn < 0 ? -yyn : 0;
; 1556 :                yyx < (int) (sizeof (yytname) / sizeof (TCHAR* ));
; 1557 :                yyx++)
; 1558 :             if (yycheck[yyx + yyn] == yyx && yyx != YYTERROR)
; 1559 :               {
; 1560 :             const TCHAR* yyq = ! yycount ? _T(", expecting ") : _T(" or ");
; 1561 :             yyp = yystpcpy (yyp, yyq);
; 1562 :             yyp = yystpcpy (yyp, yytname[yyx]);
; 1563 :             yycount++;
; 1564 :               }
; 1565 :         }
; 1566 :           yyerror (yymsg);
; 1567 :           YYSTACK_FREE (yymsg);
; 1568 :         }
; 1569 :       else
; 1570 :         yyerror (_T("syntax error; also virtual memory exhausted"));
; 1571 :     }
; 1572 :       else
; 1573 : #endif /* YYERROR_VERBOSE */
; 1574 :     yyerror (_T("syntax error"));

  00742	68 00 00 00 00	 push	 OFFSET ??_C@_1BK@ECDIFIKG@?$AAs?$AAy?$AAn?$AAt?$AAa?$AAx?$AA?5?$AAe?$AAr?$AAr?$AAo?$AAr?$AA?$AA@
  00747	e8 00 00 00 00	 call	 ?yyerror@@YAXPB_W@Z	; yyerror
  0074c	83 c4 04	 add	 esp, 4
$LN22@yyparse:

; 1575 :     }
; 1576 : 
; 1577 : 
; 1578 : 
; 1579 :   if (yyerrstatus == 3)

  0074f	83 bd 1c fb ff
	ff 03		 cmp	 DWORD PTR _yyerrstatus$[ebp], 3
  00756	0f 85 8e 00 00
	00		 jne	 $yyerrlab2$138298

; 1580 :     {
; 1581 :       /* If just tried and failed to reuse lookahead token after an
; 1582 :      error, discard it.  */
; 1583 : 
; 1584 :       /* Return failure if at end of input.  */
; 1585 :       if (yychar == YYEOF)

  0075c	83 3d 00 00 00
	00 00		 cmp	 DWORD PTR ?yychar@@3HA, 0 ; yychar
  00763	75 67		 jne	 SHORT $LN20@yyparse

; 1586 :         {
; 1587 :       /* Pop the error token.  */
; 1588 :           YYPOPSTACK;

  00765	8b 45 f8	 mov	 eax, DWORD PTR _yyvsp$[ebp]
  00768	83 e8 04	 sub	 eax, 4
  0076b	89 45 f8	 mov	 DWORD PTR _yyvsp$[ebp], eax
  0076e	8b 8d 2c fb ff
	ff		 mov	 ecx, DWORD PTR _yyssp$[ebp]
  00774	83 e9 02	 sub	 ecx, 2
  00777	89 8d 2c fb ff
	ff		 mov	 DWORD PTR _yyssp$[ebp], ecx
$LN19@yyparse:

; 1589 :       /* Pop the rest of the stack.  */
; 1590 :       while (yyss < yyssp)

  0077d	8b 95 c8 fc ff
	ff		 mov	 edx, DWORD PTR _yyss$[ebp]
  00783	3b 95 2c fb ff
	ff		 cmp	 edx, DWORD PTR _yyssp$[ebp]
  00789	73 37		 jae	 SHORT $LN18@yyparse

; 1591 :         {
; 1592 :           YYDSYMPRINTF (_T("Error: popping"), yystos[*yyssp], yyvsp, yylsp);
; 1593 :           yydestruct (yystos[*yyssp], yyvsp);

  0078b	8b 45 f8	 mov	 eax, DWORD PTR _yyvsp$[ebp]
  0078e	50		 push	 eax
  0078f	8b 8d 2c fb ff
	ff		 mov	 ecx, DWORD PTR _yyssp$[ebp]
  00795	0f bf 11	 movsx	 edx, WORD PTR [ecx]
  00798	0f b6 82 00 00
	00 00		 movzx	 eax, BYTE PTR _yystos[edx]
  0079f	50		 push	 eax
  007a0	e8 00 00 00 00	 call	 ?yydestruct@@YAXHPATYYSTYPE@@@Z ; yydestruct
  007a5	83 c4 08	 add	 esp, 8

; 1594 :           YYPOPSTACK;

  007a8	8b 4d f8	 mov	 ecx, DWORD PTR _yyvsp$[ebp]
  007ab	83 e9 04	 sub	 ecx, 4
  007ae	89 4d f8	 mov	 DWORD PTR _yyvsp$[ebp], ecx
  007b1	8b 95 2c fb ff
	ff		 mov	 edx, DWORD PTR _yyssp$[ebp]
  007b7	83 ea 02	 sub	 edx, 2
  007ba	89 95 2c fb ff
	ff		 mov	 DWORD PTR _yyssp$[ebp], edx

; 1595 :         }

  007c0	eb bb		 jmp	 SHORT $LN19@yyparse
$LN18@yyparse:

; 1596 :       YYABORT;

  007c2	e9 39 01 00 00	 jmp	 $yyabortlab$138232
  007c7	e9 34 01 00 00	 jmp	 $yyabortlab$138232
$LN20@yyparse:

; 1597 :         }
; 1598 : 
; 1599 :       YYDSYMPRINTF (_T("Error: discarding"), yytoken, &yylval, &yylloc);
; 1600 :       yydestruct (yytoken, &yylval);

  007cc	68 00 00 00 00	 push	 OFFSET ?yylval@@3TYYSTYPE@@A ; yylval
  007d1	8b 85 d4 fc ff
	ff		 mov	 eax, DWORD PTR _yytoken$[ebp]
  007d7	50		 push	 eax
  007d8	e8 00 00 00 00	 call	 ?yydestruct@@YAXHPATYYSTYPE@@@Z ; yydestruct
  007dd	83 c4 08	 add	 esp, 8

; 1601 :       yychar = YYEMPTY;

  007e0	c7 05 00 00 00
	00 fe ff ff ff	 mov	 DWORD PTR ?yychar@@3HA, -2 ; yychar, fffffffeH
$yyerrlab2$138298:

; 1602 : 
; 1603 :     }
; 1604 : 
; 1605 :   /* Else will try to reuse lookahead token after shifting the error
; 1606 :      token.  */
; 1607 :   goto yyerrlab2;
; 1608 : 
; 1609 : 
; 1610 : /*----------------------------------------------------.
; 1611 : | yyerrlab1 -- error raised explicitly by an action.  |
; 1612 : `----------------------------------------------------*/
; 1613 : //yyerrlab1:
; 1614 : 
; 1615 :   /* Suppress GCC warning that yyerrlab1 is unused when no action
; 1616 :      invokes YYERROR.  */
; 1617 : #if defined (__GNUC_MINOR__) && 2093 <= (__GNUC__ * 1000 + __GNUC_MINOR__) \
; 1618 :     && !defined __cplusplus
; 1619 :   __attribute__ ((__unused__))
; 1620 : #endif
; 1621 : 
; 1622 : 
; 1623 :   goto yyerrlab2;
; 1624 : 
; 1625 : 
; 1626 : /*---------------------------------------------------------------.
; 1627 : | yyerrlab2 -- pop states until the error token can be shifted.  |
; 1628 : `---------------------------------------------------------------*/
; 1629 : yyerrlab2:
; 1630 :   yyerrstatus = 3;    /* Each real token shifted decrements this.  */

  007ea	c7 85 1c fb ff
	ff 03 00 00 00	 mov	 DWORD PTR _yyerrstatus$[ebp], 3
$LN15@yyparse:

; 1631 : 
; 1632 :   for (;;)
; 1633 :     {
; 1634 :       yyn = yypact[yystate];

  007f4	8b 8d 28 fb ff
	ff		 mov	 ecx, DWORD PTR _yystate$[ebp]
  007fa	0f bf 14 4d 00
	00 00 00	 movsx	 edx, WORD PTR _yypact[ecx*2]
  00802	89 95 20 fb ff
	ff		 mov	 DWORD PTR _yyn$[ebp], edx

; 1635 :       if (yyn != YYPACT_NINF)

  00808	81 bd 20 fb ff
	ff 20 ff ff ff	 cmp	 DWORD PTR _yyn$[ebp], -224 ; ffffff20H
  00812	74 4f		 je	 SHORT $LN13@yyparse

; 1636 :     {
; 1637 :       yyn += YYTERROR;

  00814	8b 85 20 fb ff
	ff		 mov	 eax, DWORD PTR _yyn$[ebp]
  0081a	83 c0 01	 add	 eax, 1
  0081d	89 85 20 fb ff
	ff		 mov	 DWORD PTR _yyn$[ebp], eax

; 1638 :       if (0 <= yyn && yyn <= YYLAST && yycheck[yyn] == YYTERROR)

  00823	78 3e		 js	 SHORT $LN13@yyparse
  00825	81 bd 20 fb ff
	ff 2e 01 00 00	 cmp	 DWORD PTR _yyn$[ebp], 302 ; 0000012eH
  0082f	7f 32		 jg	 SHORT $LN13@yyparse
  00831	8b 8d 20 fb ff
	ff		 mov	 ecx, DWORD PTR _yyn$[ebp]
  00837	0f bf 14 4d 00
	00 00 00	 movsx	 edx, WORD PTR _yycheck[ecx*2]
  0083f	83 fa 01	 cmp	 edx, 1
  00842	75 1f		 jne	 SHORT $LN13@yyparse

; 1639 :         {
; 1640 :           yyn = yytable[yyn];

  00844	8b 85 20 fb ff
	ff		 mov	 eax, DWORD PTR _yyn$[ebp]
  0084a	0f bf 0c 45 00
	00 00 00	 movsx	 ecx, WORD PTR _yytable[eax*2]
  00852	89 8d 20 fb ff
	ff		 mov	 DWORD PTR _yyn$[ebp], ecx

; 1641 :           if (0 < yyn)

  00858	83 bd 20 fb ff
	ff 00		 cmp	 DWORD PTR _yyn$[ebp], 0
  0085f	7e 02		 jle	 SHORT $LN13@yyparse

; 1642 :         break;

  00861	eb 5e		 jmp	 SHORT $LN14@yyparse
$LN13@yyparse:

; 1643 :         }
; 1644 :     }
; 1645 : 
; 1646 :       /* Pop the current state because it cannot handle the error token.  */
; 1647 :       if (yyssp == yyss)

  00863	8b 95 2c fb ff
	ff		 mov	 edx, DWORD PTR _yyssp$[ebp]
  00869	3b 95 c8 fc ff
	ff		 cmp	 edx, DWORD PTR _yyss$[ebp]
  0086f	75 0a		 jne	 SHORT $LN10@yyparse
  00871	e9 8a 00 00 00	 jmp	 $yyabortlab$138232

; 1648 :     YYABORT;

  00876	e9 85 00 00 00	 jmp	 $yyabortlab$138232
$LN10@yyparse:

; 1649 : 
; 1650 :       YYDSYMPRINTF (_T("Error: popping"), yystos[*yyssp], yyvsp, yylsp);
; 1651 :       yydestruct (yystos[yystate], yyvsp);

  0087b	8b 45 f8	 mov	 eax, DWORD PTR _yyvsp$[ebp]
  0087e	50		 push	 eax
  0087f	8b 8d 28 fb ff
	ff		 mov	 ecx, DWORD PTR _yystate$[ebp]
  00885	0f b6 91 00 00
	00 00		 movzx	 edx, BYTE PTR _yystos[ecx]
  0088c	52		 push	 edx
  0088d	e8 00 00 00 00	 call	 ?yydestruct@@YAXHPATYYSTYPE@@@Z ; yydestruct
  00892	83 c4 08	 add	 esp, 8

; 1652 :       yyvsp--;

  00895	8b 45 f8	 mov	 eax, DWORD PTR _yyvsp$[ebp]
  00898	83 e8 04	 sub	 eax, 4
  0089b	89 45 f8	 mov	 DWORD PTR _yyvsp$[ebp], eax

; 1653 :       yystate = *--yyssp;

  0089e	8b 8d 2c fb ff
	ff		 mov	 ecx, DWORD PTR _yyssp$[ebp]
  008a4	83 e9 02	 sub	 ecx, 2
  008a7	89 8d 2c fb ff
	ff		 mov	 DWORD PTR _yyssp$[ebp], ecx
  008ad	8b 95 2c fb ff
	ff		 mov	 edx, DWORD PTR _yyssp$[ebp]
  008b3	0f bf 02	 movsx	 eax, WORD PTR [edx]
  008b6	89 85 28 fb ff
	ff		 mov	 DWORD PTR _yystate$[ebp], eax

; 1654 : 
; 1655 :       YY_STACK_PRINT (yyss, yyssp);
; 1656 :     }

  008bc	e9 33 ff ff ff	 jmp	 $LN15@yyparse
$LN14@yyparse:

; 1657 : 
; 1658 :   if (yyn == YYFINAL)

  008c1	83 bd 20 fb ff
	ff 0c		 cmp	 DWORD PTR _yyn$[ebp], 12 ; 0000000cH
  008c8	75 04		 jne	 SHORT $LN8@yyparse
  008ca	eb 26		 jmp	 SHORT $yyacceptlab$138254

; 1659 :     YYACCEPT;

  008cc	eb 24		 jmp	 SHORT $yyacceptlab$138254
$LN8@yyparse:

; 1660 : 
; 1661 :   YYDPRINTF ((stderr, _T("Shifting error token, ")));
; 1662 : 
; 1663 :   *++yyvsp = yylval;

  008ce	8b 4d f8	 mov	 ecx, DWORD PTR _yyvsp$[ebp]
  008d1	83 c1 04	 add	 ecx, 4
  008d4	89 4d f8	 mov	 DWORD PTR _yyvsp$[ebp], ecx
  008d7	8b 55 f8	 mov	 edx, DWORD PTR _yyvsp$[ebp]
  008da	a1 00 00 00 00	 mov	 eax, DWORD PTR ?yylval@@3TYYSTYPE@@A ; yylval
  008df	89 02		 mov	 DWORD PTR [edx], eax

; 1664 : 
; 1665 : 
; 1666 :   yystate = yyn;

  008e1	8b 8d 20 fb ff
	ff		 mov	 ecx, DWORD PTR _yyn$[ebp]
  008e7	89 8d 28 fb ff
	ff		 mov	 DWORD PTR _yystate$[ebp], ecx
  008ed	e9 8f f7 ff ff	 jmp	 $yynewstate$138188
$yyacceptlab$138254:

; 1667 :   goto yynewstate;
; 1668 : 
; 1669 : 
; 1670 : /*-------------------------------------.
; 1671 : | yyacceptlab -- YYACCEPT comes here.  |
; 1672 : `-------------------------------------*/
; 1673 : yyacceptlab:
; 1674 :   yyresult = 0;

  008f2	c7 85 24 fb ff
	ff 00 00 00 00	 mov	 DWORD PTR _yyresult$[ebp], 0
  008fc	eb 27		 jmp	 SHORT $yyreturn$138310
  008fe	eb 25		 jmp	 SHORT $yyreturn$138310
$yyabortlab$138232:

; 1675 :   goto yyreturn;
; 1676 : 
; 1677 : /*-----------------------------------.
; 1678 : | yyabortlab -- YYABORT comes here.  |
; 1679 : `-----------------------------------*/
; 1680 : yyabortlab:
; 1681 :   yyresult = 1;

  00900	c7 85 24 fb ff
	ff 01 00 00 00	 mov	 DWORD PTR _yyresult$[ebp], 1
  0090a	eb 19		 jmp	 SHORT $yyreturn$138310
  0090c	eb 17		 jmp	 SHORT $yyreturn$138310
$yyoverflowlab$138192:

; 1682 :   goto yyreturn;
; 1683 : 
; 1684 : #ifndef yyoverflow
; 1685 : /*----------------------------------------------.
; 1686 : | yyoverflowlab -- parser overflow comes here.  |
; 1687 : `----------------------------------------------*/
; 1688 : yyoverflowlab:
; 1689 :   yyerror (_T("parser stack overflow"));

  0090e	68 00 00 00 00	 push	 OFFSET ??_C@_1CM@BIEIIFPA@?$AAp?$AAa?$AAr?$AAs?$AAe?$AAr?$AA?5?$AAs?$AAt?$AAa?$AAc?$AAk?$AA?5?$AAo?$AAv?$AAe?$AAr?$AAf?$AAl?$AAo?$AAw?$AA?$AA@
  00913	e8 00 00 00 00	 call	 ?yyerror@@YAXPB_W@Z	; yyerror
  00918	83 c4 04	 add	 esp, 4

; 1690 :   yyresult = 2;

  0091b	c7 85 24 fb ff
	ff 02 00 00 00	 mov	 DWORD PTR _yyresult$[ebp], 2
$yyreturn$138310:

; 1691 :   /* Fall through.  */
; 1692 : #endif
; 1693 : 
; 1694 : yyreturn:
; 1695 : #ifndef yyoverflow
; 1696 :   if (yyss != yyssa)

  00925	8b 95 c8 fc ff
	ff		 mov	 edx, DWORD PTR _yyss$[ebp]
  0092b	8d 85 30 fb ff
	ff		 lea	 eax, DWORD PTR _yyssa$[ebp]
  00931	3b d0		 cmp	 edx, eax
  00933	74 04		 je	 SHORT $LN4@yyparse
$LN2@yyparse:

; 1697 :     YYSTACK_FREE (yyss);

  00935	33 c9		 xor	 ecx, ecx
  00937	75 fc		 jne	 SHORT $LN2@yyparse
$LN4@yyparse:

; 1698 : #endif
; 1699 :   return yyresult;

  00939	8b 85 24 fb ff
	ff		 mov	 eax, DWORD PTR _yyresult$[ebp]

; 1700 : }

  0093f	8d a5 f0 fa ff
	ff		 lea	 esp, DWORD PTR [ebp-1296]
  00945	5e		 pop	 esi
  00946	8b 8d c0 fc ff
	ff		 mov	 ecx, DWORD PTR __$ArrayPad$[ebp]
  0094c	33 cd		 xor	 ecx, ebp
  0094e	e8 00 00 00 00	 call	 @__security_check_cookie@4
  00953	8b e5		 mov	 esp, ebp
  00955	5d		 pop	 ebp
  00956	c3		 ret	 0
  00957	90		 npad	 1
$LN107@yyparse:
  00958	00 00 00 00	 DD	 $LN47@yyparse
  0095c	00 00 00 00	 DD	 $LN46@yyparse
  00960	00 00 00 00	 DD	 $LN45@yyparse
  00964	00 00 00 00	 DD	 $LN44@yyparse
  00968	00 00 00 00	 DD	 $LN43@yyparse
  0096c	00 00 00 00	 DD	 $LN42@yyparse
  00970	00 00 00 00	 DD	 $LN41@yyparse
  00974	00 00 00 00	 DD	 $LN40@yyparse
  00978	00 00 00 00	 DD	 $LN39@yyparse
  0097c	00 00 00 00	 DD	 $LN38@yyparse
  00980	00 00 00 00	 DD	 $LN37@yyparse
  00984	00 00 00 00	 DD	 $LN36@yyparse
  00988	00 00 00 00	 DD	 $LN35@yyparse
  0098c	00 00 00 00	 DD	 $LN34@yyparse
  00990	00 00 00 00	 DD	 $LN33@yyparse
  00994	00 00 00 00	 DD	 $LN32@yyparse
  00998	00 00 00 00	 DD	 $LN30@yyparse
  0099c	00 00 00 00	 DD	 $LN29@yyparse
  009a0	00 00 00 00	 DD	 $LN28@yyparse
  009a4	00 00 00 00	 DD	 $LN27@yyparse
  009a8	00 00 00 00	 DD	 $LN26@yyparse
  009ac	00 00 00 00	 DD	 $LN25@yyparse
  009b0	00 00 00 00	 DD	 $LN48@yyparse
$LN106@yyparse:
  009b4	00		 DB	 0
  009b5	16		 DB	 22			; 00000016H
  009b6	16		 DB	 22			; 00000016H
  009b7	16		 DB	 22			; 00000016H
  009b8	16		 DB	 22			; 00000016H
  009b9	16		 DB	 22			; 00000016H
  009ba	16		 DB	 22			; 00000016H
  009bb	01		 DB	 1
  009bc	02		 DB	 2
  009bd	16		 DB	 22			; 00000016H
  009be	16		 DB	 22			; 00000016H
  009bf	16		 DB	 22			; 00000016H
  009c0	16		 DB	 22			; 00000016H
  009c1	16		 DB	 22			; 00000016H
  009c2	16		 DB	 22			; 00000016H
  009c3	16		 DB	 22			; 00000016H
  009c4	16		 DB	 22			; 00000016H
  009c5	16		 DB	 22			; 00000016H
  009c6	16		 DB	 22			; 00000016H
  009c7	16		 DB	 22			; 00000016H
  009c8	16		 DB	 22			; 00000016H
  009c9	03		 DB	 3
  009ca	04		 DB	 4
  009cb	16		 DB	 22			; 00000016H
  009cc	16		 DB	 22			; 00000016H
  009cd	16		 DB	 22			; 00000016H
  009ce	16		 DB	 22			; 00000016H
  009cf	16		 DB	 22			; 00000016H
  009d0	16		 DB	 22			; 00000016H
  009d1	16		 DB	 22			; 00000016H
  009d2	16		 DB	 22			; 00000016H
  009d3	16		 DB	 22			; 00000016H
  009d4	16		 DB	 22			; 00000016H
  009d5	16		 DB	 22			; 00000016H
  009d6	16		 DB	 22			; 00000016H
  009d7	16		 DB	 22			; 00000016H
  009d8	16		 DB	 22			; 00000016H
  009d9	16		 DB	 22			; 00000016H
  009da	16		 DB	 22			; 00000016H
  009db	16		 DB	 22			; 00000016H
  009dc	16		 DB	 22			; 00000016H
  009dd	16		 DB	 22			; 00000016H
  009de	16		 DB	 22			; 00000016H
  009df	16		 DB	 22			; 00000016H
  009e0	16		 DB	 22			; 00000016H
  009e1	16		 DB	 22			; 00000016H
  009e2	16		 DB	 22			; 00000016H
  009e3	16		 DB	 22			; 00000016H
  009e4	16		 DB	 22			; 00000016H
  009e5	16		 DB	 22			; 00000016H
  009e6	16		 DB	 22			; 00000016H
  009e7	16		 DB	 22			; 00000016H
  009e8	16		 DB	 22			; 00000016H
  009e9	16		 DB	 22			; 00000016H
  009ea	16		 DB	 22			; 00000016H
  009eb	16		 DB	 22			; 00000016H
  009ec	16		 DB	 22			; 00000016H
  009ed	16		 DB	 22			; 00000016H
  009ee	16		 DB	 22			; 00000016H
  009ef	16		 DB	 22			; 00000016H
  009f0	16		 DB	 22			; 00000016H
  009f1	16		 DB	 22			; 00000016H
  009f2	16		 DB	 22			; 00000016H
  009f3	16		 DB	 22			; 00000016H
  009f4	16		 DB	 22			; 00000016H
  009f5	16		 DB	 22			; 00000016H
  009f6	16		 DB	 22			; 00000016H
  009f7	16		 DB	 22			; 00000016H
  009f8	16		 DB	 22			; 00000016H
  009f9	16		 DB	 22			; 00000016H
  009fa	16		 DB	 22			; 00000016H
  009fb	16		 DB	 22			; 00000016H
  009fc	16		 DB	 22			; 00000016H
  009fd	16		 DB	 22			; 00000016H
  009fe	16		 DB	 22			; 00000016H
  009ff	16		 DB	 22			; 00000016H
  00a00	16		 DB	 22			; 00000016H
  00a01	16		 DB	 22			; 00000016H
  00a02	16		 DB	 22			; 00000016H
  00a03	16		 DB	 22			; 00000016H
  00a04	16		 DB	 22			; 00000016H
  00a05	16		 DB	 22			; 00000016H
  00a06	16		 DB	 22			; 00000016H
  00a07	16		 DB	 22			; 00000016H
  00a08	16		 DB	 22			; 00000016H
  00a09	16		 DB	 22			; 00000016H
  00a0a	16		 DB	 22			; 00000016H
  00a0b	16		 DB	 22			; 00000016H
  00a0c	16		 DB	 22			; 00000016H
  00a0d	16		 DB	 22			; 00000016H
  00a0e	16		 DB	 22			; 00000016H
  00a0f	16		 DB	 22			; 00000016H
  00a10	16		 DB	 22			; 00000016H
  00a11	16		 DB	 22			; 00000016H
  00a12	16		 DB	 22			; 00000016H
  00a13	16		 DB	 22			; 00000016H
  00a14	16		 DB	 22			; 00000016H
  00a15	05		 DB	 5
  00a16	06		 DB	 6
  00a17	07		 DB	 7
  00a18	16		 DB	 22			; 00000016H
  00a19	08		 DB	 8
  00a1a	16		 DB	 22			; 00000016H
  00a1b	16		 DB	 22			; 00000016H
  00a1c	16		 DB	 22			; 00000016H
  00a1d	16		 DB	 22			; 00000016H
  00a1e	16		 DB	 22			; 00000016H
  00a1f	16		 DB	 22			; 00000016H
  00a20	16		 DB	 22			; 00000016H
  00a21	16		 DB	 22			; 00000016H
  00a22	16		 DB	 22			; 00000016H
  00a23	09		 DB	 9
  00a24	0a		 DB	 10			; 0000000aH
  00a25	0b		 DB	 11			; 0000000bH
  00a26	0c		 DB	 12			; 0000000cH
  00a27	0d		 DB	 13			; 0000000dH
  00a28	0e		 DB	 14			; 0000000eH
  00a29	0f		 DB	 15			; 0000000fH
  00a2a	16		 DB	 22			; 00000016H
  00a2b	10		 DB	 16			; 00000010H
  00a2c	11		 DB	 17			; 00000011H
  00a2d	12		 DB	 18			; 00000012H
  00a2e	13		 DB	 19			; 00000013H
  00a2f	14		 DB	 20			; 00000014H
  00a30	15		 DB	 21			; 00000015H
?yyparse@@YAHXZ ENDP					; yyparse
END
